:020000040800F2
:10000000105C0020E10100088D4E0008693A0008EC
:10001000C1460008010A0008455F00080000000012
:10002000000000000000000000000000490100087E
:10003000FD0A0008000000008D0100080D570008AF
:10004000FB010008FB010008FB010008FB010008A0
:10005000FB010008FB010008FB010008FB01000890
:10006000FB010008FB010008FB010008FB01000880
:10007000FB010008A10A0008B10A0008C10A000833
:10008000FB010008FB010008D9070008FB0100087C
:10009000FB010008FB010008FB010008FB01000850
:1000A000FB010008FB010008FB010008FB01000840
:1000B000C1570008DD570008FB010008FB010008DC
:1000C000FB010008FB010008FB010008FB01000820
:1000D000FB010008A15E0008FB010008355F000875
:1000E000FB010008FB010008FB010008FB01000800
:1000F000FB010008FB010008FB010008FB010008F0
:10010000FB010008FB010008FB010008FB010008DF
:10011000FB010008FB010008FB010008FB010008CF
:10012000FB010008FB010008FB010008FB010008BF
:10013000DFF810D000F004FB004800478569000894
:10014000AFF30080105C0020224B19680868B0E80B
:10015000F00F80F30988BFF36F8F4FF0000080F33A
:1001600011884EF00D0E7047000000000648006830
:10017000006880F3088862B661B6BFF34F8FBFF3A3
:100180006F8F00DF00BF00BF08ED00E0EFF30980D4
:10019000BFF36F8F0F4B1A6820E9F00F106008B59E
:1001A0004FF0500080F31188BFF34F8FBFF36F8F74
:1001B00007F02AFC4FF0000080F31188BDE80840EA
:1001C00019680868B0E8F00F80F30988BFF36F8FF3
:1001D000704700BFB0050020EFF3058070470000B6
:1001E0000648804706480047FEE7FEE7FEE7FEE7D1
:1001F000FEE7FEE7FEE7FEE7FEE7FEE7BF57000883
:1002000031010008202A04DB203A21FA02F0002103
:10021000704721FA02F3D040C2F120029140084316
:100220001946704740EA01039B0703D009E008C95B
:10023000121F08C0042AFAD203E011F8013B00F8AB
:10024000013B521EF9D27047D2B201E000F8012BF7
:10025000491EFBD270470022F6E710B513460A4646
:1002600004461946FFF7F0FF204610BD421C10F867
:10027000011B0029FBD1801A7047F0B480EA01020B
:10028000D40F4200B2EB410F02D20246084611469B
:100290004A0042D0C30DDDB2C1F3C752AD1A202DC2
:1002A00035DAC1F3160141F4000204B15242C5F13E
:1002B000200602FA06F12A411044B3EBD05F23D0A6
:1002C000C4B1012DA0EBC35009DCF0BC4FF00042DB
:1002D00002EAC352DBB200F5000000F0A6B940000C
:1002E00000F1807000EBC350A0F1807040EAD17043
:1002F000490009E0490841EAC071A0EBC35000F58C
:100300000000400800EBC350F0BC00F085B961422A
:10031000012202EB4101001BF6E7F0BC704781F0BF
:100320000041AAE780F00040A7E780EA010210B58B
:1003300002F00043400022D04A001FD0010E01EB22
:100340001261C0F35600C2F3560240F4000042F4BA
:100350000002A0FB022000047F39140400D0401CDE
:1003600050EA124001D44000491EC2B20C0604EB10
:10037000D010401C4008802A02D003E0002010BDAD
:1003800020F00100002900DA0020184310BD30B42D
:1003900080EA010202F0004530F0004221F0004006
:1003A00013D090B1C30DD40DC2F31601C0F31600E3
:1003B000E41A41F4000140F400027D34914201D37B
:1003C000641C00E04900002C02DA30BC00207047B9
:1003D0004FF400000023914201D3891A03434008DF
:1003E0004FEA4101F7D151B1914202D14FF00041A2
:1003F00005E002D24FF0010101E06FF0010103EBD3
:10040000C450284430BC00F007B92DE9FE4F81EA02
:10041000030404F0004421F0004100944FF0000B6D
:1004200023F0004350EA01045ED052EA03045BD09B
:10043000C3F30A54C1F30A552C44A4F2F3340194D3
:10044000A0FB0254C1F3130141F48011C3F3130361
:1004500043F4801301FB024400FB034E840A970A15
:1004600044EA815447EA8357A4FB076802958D0A42
:1004700005FB07854FEA932C04FB0C542705029DCE
:100480004FEA065847EA1637B5EB08056EEB070C3E
:10049000870E920E47EA811742EA8312A7FB0201F8
:1004A000B6EB0B0164EB00042B0D43EA0C335E1832
:1004B00044EB1C50DA465146E7FB0201C5F3130436
:1004C0004FEA0B3343EA14534FEA0432019C43EAE8
:1004D0000603A4F10C040294009CCDE900B400F0E2
:1004E000E1F803B0BDE8F08F00200146F9E7C10F45
:1004F00080EAE0700844CA079623002100F095B80E
:1005000096230022114600F090B820F00040C10D63
:10051000C0F3160040F400007F2901DA0020704784
:10052000962903DCC1F19601C8407047963988408E
:100530007047C1F30A5210B5C1F3130140F2FF3303
:1005400041F480119A4201DA002010BD40F2334399
:100550009A42A2F2334203DC5242FFF753FE10BD2F
:10056000904010BD00F0004230F000400AD0C10DB4
:1005700001F56071C0F3160042EA0151C20840075C
:100580001143704700200146704701F0004330B42A
:1005900021F0004150EA010206D00A0DA2F5607276
:1005A000C1F31301002A02DC30BC00207047440F65
:1005B00044EAC104C100E01830BC00EBC25000F0B6
:1005C0002BB80000002801DBC0F10040002901DB4E
:1005D000C1F1004181427047002801DBC0F10040B9
:1005E000002901DBC1F100418842704730B50B465C
:1005F000014600202022012409E021FA02F59D4253
:1006000005D303FA02F5491B04FA02F52844151E26
:10061000A2F10102F1DC30BD0029A8BF7047401CE7
:10062000490008BF20F00100704710B4B0FA80FC08
:1006300000FA0CF050EA010404BF10BC704749B145
:10064000CCF1200421FA04F411FA0CF118BF0121B5
:1006500021430843A3EB0C01CB1D4FEA00614FEA95
:10066000102042BF002010BC704700EBC350104464
:100670000029A4BF10BC7047401C490008BF20F0EF
:10068000010010BC704710B5141E73F1000408DAA5
:10069000401C41F1000192185B411A4301D120F046
:1006A000010010BD2DE9F04D92469B4611B1B1FA03
:1006B00081F202E0B0FA80F22032904600F052F867
:1006C00004460F4640EA0A0041EA0B0153465A46E7
:1006D000084313D0114653EA010019D0C8F1400273
:1006E0005046FFF78FFD05460E4650465946424696
:1006F00000F038F8084305D0012004E020463946D0
:10070000BDE8F08D0020054346EAE0762C433743F0
:100710000A986305E40AA0EB08000022FD0A44EAF7
:1007200047540A3002D500200146E9E701051019B7
:100730006941DDE9084500196941BDE8F04DA2E7CE
:10074000064C074D06E0E06840F0010394E807001E
:1007500098471034AC42F6D3FFF7EEFC0C8000084B
:100760002C800008202A04DB203A00FA02F1002045
:1007700070479140C2F1200320FA03F319439040DF
:10078000704770B58C1810F8015B15F0070301D1A4
:1007900010F8013B2A1106D110F8012B03E010F8E4
:1007A000016B01F8016B5B1EF9D12B0705D4002307
:1007B000521E0DD401F8013BFAE710F8013BCB1AA9
:1007C000921C03E013F8015B01F8015B521EF9D59E
:1007D000A142D8D3002070BD10B5024800F05FFCE4
:1007E00010BD0000540F002070B50446002520689D
:1007F000806800F0010018B32068806820F00100D4
:100800002168886001F040FD054613E001F03CFDE1
:10081000401B02280ED92068806800F0010048B112
:10082000A06A40F01000A062E06A40F00100E062BF
:10083000012070BD2068806800F001000028E5D12B
:100840000020F6E738B50446002500200090206817
:10085000806800F0010078BB2068806840F00100EB
:1008600021688860194800681949B0FBF1F00090D0
:1008700002E00098401E009000980028F9D101F095
:1008800003FD054619E001F0FFFC401B022814D9C6
:100890002068806800F0010078B9A06A40F010007C
:1008A000A062E06A40F00100E06200BF002084F82E
:1008B000240000BF012038BD05E02068806800F0FA
:1008C00001000028DFD00020F5E70000AC05002083
:1008D00040420F0010B5184806F048FC1749088040
:1008E000174806F043FC17490880144800884FF663
:1008F000FF71884202D01148008801E01248008848
:10090000114908800F4800884FF6FF71884202D0D5
:100910000C48008801E00D4800880C4908800A480E
:100920000088C0F30E000849088008480088C0F31A
:100930000E000649088010BD00180708740000204A
:100940000020070876000020860000208800002094
:10095000F0B597B006460D4601A803F0B5F800249F
:1009600012E004F50070854202D94FF4007700E0F0
:100970002F1B31193A461148FFF754FC3A460F49EC
:1009800001A803F0A1FC3C44AC42EAD301A90C4805
:1009900003F06CF8002407E00948005D0949615C38
:1009A000884200D002E0641C102CF5D300BF102C4C
:1009B00002D3012017B0F0BD0020FBE7002000208B
:1009C0001E28002000500708F0B50446187822F8C9
:1009D00010400025002004E032F810603544461C29
:1009E000F0B20A28F8DB0A20B5FBF0F0088018788E
:1009F000401C0A2690FBF6F706FB17001870F0BDA6
:100A000000BFFEE72DE9FC4707460D463846FFF7D5
:100A100077FD81462946FFF788FC04464FF08B415D
:100A2000FFF7B5FC064631462846FFF778FC8146BD
:100A300049463046FFF7ABFC04461549FFF775FC05
:100A40008046002419E0134A601C52F820104046EA
:100A5000FFF7C2FD10D80F4850F824104046FFF7AA
:100A6000B1FD09D20A2023460A4A0B49CDE90040CC
:100A7000404605F0E1FD04E0641C40F2472084425A
:100A8000E1D300BF05480088FFF73AFDBDE8FC87C9
:100A900000002041D40200208C000020200500200E
:100AA00010B5024800F0F2FE10BD00009048002092
:100AB00010B5024800F0EAFE10BD00004C480020CE
:100AC00010B5024800F0E2FE10BD0000084800200A
:100AD00030B590F840500124AC40C56B6C600468A0
:100AE00063604468102C04D10468A2600468E1606B
:100AF00003E00468A1600468E26030BD704770B52F
:100B000003460024002010E00E5C451C4D5D46EAC3
:100B10000526851C4D5D46EA0546C51C4D5D46EA29
:100B2000056543F82450641C001D9042ECD370BD51
:100B300070B5034614460022002015E011F822503B
:100B40001D5431F82250C5F30726451C5E5551F857
:100B50002250C5F30746851C5E5551F822502D0ED4
:100B6000C61C9D55521C001DA042E7D370BD72B635
:100B700000BFFEE70021074AD1610749096941F03A
:100B80000401054A11611146096941F040011161F2
:100B900070470000C00F0020002002400021074ADB
:100BA000D1610749096941F00201054A1161114605
:100BB0004861096941F0400111617047C00F002090
:100BC000002002400022054BDA61054A126942F01A
:100BD0000102034B1A61018070470000C00F002022
:100BE0000020024000201E49C96801F0100139B1FF
:100BF0001C49C96941F002011A4AD16140F0100054
:100C00001749C96801F0040139B11649C96941F0B1
:100C10000101144AD16140F004001149C96901F091
:100C2000010169B10F49C96941F004010D4AD1615F
:100C300000BF0B49C96921F00101094AD16100BF18
:100C400000BF40F20111884206D10549C96921F06F
:100C50000101034AD16101E00149C86000BF70474A
:100C600000200240C00F002070B5044601F00CFBCC
:100C7000054609E0601C38B124B101F005FB401BBA
:100C8000A04201D9032070BD1248C06800F00100E5
:100C90000028EFD10F48C06800F0200020B100BF4D
:100CA00020200C49C86000BF0A48C06800F010004E
:100CB00048B90848C06900F0010020B90548C0687B
:100CC00000F0040018B1FFF78DFF0120DBE70020E2
:100CD000D9E7000000200240F0B503461C4600257D
:100CE0000026084607E010F8015B10F8016B45EAA2
:100CF000062724F8027B171EA2F1010C1FFA8CF2C2
:100D0000F1D1F0BD2DE9F04786B080460E46914600
:100D10004FF0000A00270025C6F30A0AA6EB0A07CF
:100D2000002005900190039701200490820239462B
:100D30001548FFF7D1FF00BF07E038F8150005EBB5
:100D40005A01114A22F811006D1C4D45F5D301F0EE
:100D5000CBF805A901A801F00DF800240BE00A4822
:100D600030F814C007EB440162460023012001F073
:100D700063F8601C84B2B4F5806FF0DB01F052F8C8
:100D800006B0BDE8F0870000001000202DE9F04714
:100D900081463A4800F0BEFB6421384800F0FAFA78
:100DA000364800F078F986B235493046FFF72AFE1A
:100DB0008046FFF7AAFB87B2324B334A33493846A5
:100DC000FFF702FE2D4800F0A5FB64212B4800F040
:100DD000E1FA2A4800F05FF985B22D480580B5B1E7
:100DE0002C48008800F4004010B12B48008802E035
:100DF000294800884042284485B240F68B60274944
:100E0000088008460088854201DB08460588244B97
:100E1000244A25492846FFF7D7FD184800F07AFBF9
:100E20006421164800F0B6FA144800F034F984B290
:100E30001E480480B4B11E48008800F4004010B180
:100E40001C48008802E01B4800884042204484B2CD
:100E500040F68B601849088008460088844201DB10
:100E600008460488154B164A16492046FFF7ACFD84
:100E7000024800F0E7FBBDE8F0870000540F0020B7
:100E8000333353407E000020840F00207800002080
:100E90008200002074000020860000201C05002035
:100EA0007F000020980F00207A000020840000209E
:100EB00076000020880000201E0500208000002011
:100EC000AC0F00207C0000202DE9F041002500241B
:100ED0001EE0002600270CE0104A02EBC4029188B5
:100EE0000E4A52F8340004F089FA304486B2781C75
:100EF000C7B20A2FF0DB052E04DB0120A0402843F7
:100F0000C5B203E00020A0402843C5B2601CC4B2B3
:100F1000082CDEDB2846BDE8F0810000F47E0008E6
:100F200002490968C1F3C300704700000C0C01407E
:100F30007047000038B5024600230020009000BF33
:100F400092F82400012801D1022038BD012082F846
:100F5000240000BF4868072812D21068406B0C7943
:100F6000641E04EB84051F24AC40A0430D796D1E64
:100F700005EB85050C68AC4020431468606327E0EE
:100F800048680D2812D21068006B0C79E41F04EB3E
:100F900084051F24AC40A0430D79ED1F05EB8505AA
:100FA0000C68AC4020431468206311E01068C06AEC
:100FB0000C790D3C04EB84051F24AC40A0430D7953
:100FC0000D3D05EB85050C68AC4020431468E062DC
:100FD00008680A2812D31068C0680C780A3C04EB31
:100FE00044050724AC40A0430D780A3D05EB4505B8
:100FF0008C68AC4020431468E0600FE01068006922
:101000000C7804EB44050724AC40A0430D7805EBB5
:1010100045058C68AC40204314682061086810289E
:1010200002D00868112827D1174C1068A0421ED1A1
:101030001068806800F40000F0B91068806840F41F
:1010400000001468A0600868102815D10F480068D7
:101050000F4CB0FBF4F000EB80004000009002E089
:101060000098401E009000980028F9D104E0906A92
:1010700040F020009062012300BF002082F824008D
:1010800000BF184661E7000000240140AC050020C5
:1010900040420F00704701460868C06C704770B549
:1010A0000446206805682068466806F0200020286D
:1010B0002DD105F00200022829D1A06A00F010000D
:1010C00018B9A06A40F40070A0622068806800F43B
:1010D0006020B0F5602F13D1207B88B9206840686C
:1010E00020F0200021684860A06A20F48070A0628F
:1010F000A06A00F4805018B9A06A40F00100A06214
:101100002046FFF7C7FF6FF012002168086006F065
:101110008000802839D105F00400042835D1A06A68
:1011200000F0100018B9A06A40F40050A0622068D6
:10113000806800F4E040B0F5E04F0DD020684068D2
:1011400000F48060D0B92068806800F46020B0F5B9
:10115000602F13D1207B88B92068406820F0800080
:1011600021684860A06A20F48050A062A06A00F460
:10117000807018B9A06A40F00100A0622046FFF715
:10118000D7FE6FF00C002168086006F04000402890
:101190000DD105F0010050B1A06A40F48030A0628A
:1011A000204600F0B5F86FF001002168086070BDBE
:1011B0002DE9F0410446002700250026A84614B971
:1011C0000120BDE8F081A06810B1207D00B100BF12
:1011D000A06A30B90020E06284F82400204600F0C4
:1011E00099F82046FFF700FB0746A06A00F01000C0
:1011F000002873D1002F7ED1A06A20F4885040F0DF
:101200000200A0623F4AD4E90001904208D1E0699F
:10121000B0F5402F02D14FF4002002E0E06900E079
:10122000E0690143207B41EA40000643A068B0F535
:10123000807F02D0A068012802D14FF4807000E0C6
:1012400000200543207D012811D1207B38B9A069F9
:10125000401E4FF4006141EA4030054307E0A06AB8
:1012600040F02000A062E06A40F00100E0622068E7
:10127000406820F4694028432168486020688068FD
:1012800021490840304321688860A068B0F5807F1C
:1012900002D0A068012802D14FF4807000E0002045
:1012A000B0F5807F03D1208A401E4FEA00582068A5
:1012B000C06A20F4700040EA08002168C862206813
:1012C000806812490840B04209D10020E062A06A5B
:1012D00020F0020040F00100A06211E00BE0A06AE3
:1012E00020F0020040F01000A062E06A40F001002F
:1012F000E062012704E0A06A40F01000A06201272C
:1013000038465EE7003C0140FDF7E1FFFE0E1FFF9F
:101310007047000010B586B004460020029003908C
:10132000049005901849206888422AD100BF1748C8
:10133000806940F40070154988610846806900F4AE
:101340000070019000BF00BF00BF0846806940F0F8
:10135000100088610846806900F01000019000BF0D
:1013600000BF072002900320039002A9084800F064
:10137000D3FD00220521122001F046F8122001F0D1
:1013800033F806B010BD00000024014000100240F8
:1013900000100140F8B504460D46002600200090DC
:1013A000002700F071FF06462068806800F4807016
:1013B00050B1A06A40F02000A06200BF002084F875
:1013C000240000BF0120F8BD2068406800F4807050
:1013D00020BB2068C06A00F47000F8B917E0681CF0
:1013E000A8B125B100F050FF801BA8420FD920689A
:1013F000006800F0020050B9A06A40F00400A0624A
:1014000000BF002084F8240000BF0320DBE7206831
:10141000006800F002000028E1D053E0022001F053
:1014200067F838490968B1FBF0F021680969364A64
:10143000114091B92168C9689211114069B92168B8
:101440000969324A114031B92168C96892111140C5
:1014500009B9142117E0292115E0216809692B4AEF
:10146000114021B92168C9689211114041B1216828
:101470000969274A114029B92168C968114009B989
:10148000542100E0FC2100FB01F718E0681C98B132
:1014900025B100F0F9FE801BA8420DD90098B84292
:1014A0000AD2A06A40F00400A06200BF002084F8C5
:1014B000240000BF032086E70098401C009000989D
:1014C000B842E3D36FF0120021680860A06A40F4CC
:1014D0000070A0622068806800F46020B0F5602F82
:1014E0000DD1207B58B9A06A20F48070A062A06A58
:1014F00000F4805018B9A06A40F00100A0620020FA
:1015000061E70000AC05002024499224922449128E
:101510004992240070B50446002500BF94F82400C9
:10152000012801D1022070BD012084F8240000BFF1
:101530002046FFF787F90546002D77D1A06A40F2D3
:101540000121884340F48070A0623C4920688842B1
:1015500008D13B48006800F4702008B9012002E07F
:10156000002000E0012078B1A06A20F48010A06281
:101570002068406800F4806000B3A06A20F4005046
:1015800040F48050A06219E0A06A40F48010A0628C
:101590002B49091F2068884203D0284920688842C7
:1015A00004D12748006800F4806000E0002028B1E2
:1015B000A06A20F4005040F48050A062A06A00F4B9
:1015C000805020B1E06A20F00600E06201E00020D7
:1015D000E06200BF002084F8240000BFC01E216824
:1015E00008602068806800F46020B0F5602F16D194
:1015F00012492068884208D11148006800F4702020
:1016000008B9012002E0002000E0012038B1206884
:10161000806840F4A000216888600CE006E0206843
:10162000806840F480102168886004E000BF0020DA
:1016300084F8240000BF284675E700000028014018
:101640000424014070B50446002500BF94F824002E
:10165000012801D1022070BD012084F8240000BFC0
:101660002046FFF7C1F805462DB9A06A20F488503E
:1016700040F00100A06200BF002084F8240000BFF9
:101680002846E8E70146002291F82100022808D008
:101690000420886300BF002081F8200000BF0120E3
:1016A00070470868006820F00E000B681860086832
:1016B000006820F001000B68186091F840300120AC
:1016C0009840CB6B5860012081F8210000BF0020BA
:1016D00081F8200000BF1046E2E7000070B5044624
:1016E000002594F82100022803D00420A0630125DE
:1016F000C1E02068006820F00E00216808602068C2
:10170000006820F00100216808605C492068884278
:1017100052D95A4978392068884201D1012047E0DE
:10172000564964392068884201D1102040E053496D
:1017300050392068884201D1801539E04F493C3941
:101740002068884201D1801432E04C492839206851
:10175000884202D14FF480302AE048491439206889
:10176000884202D14FF4801022E044492068884228
:1017700001D140041CE042492068884201D1012087
:1017800016E03F4914312068884201D110200FE053
:101790003B4928312068884201D1801508E038494A
:1017A0003C312068884201D1801401E04FF4803040
:1017B0003349091F086051E0304978392068884270
:1017C00001D1012047E02D4964392068884201D1C8
:1017D000102040E0294950392068884201D1801505
:1017E00039E026493C392068884201D1801432E032
:1017F000224928392068884202D14FF480302AE0FB
:101800001E4914392068884202D14FF4801022E02A
:101810001A492068884201D140041CE01849206818
:10182000884201D1012016E0154914312068884210
:1018300001D110200FE0124928312068884201D1DF
:10184000801508E00E493C312068884201D180149F
:1018500001E04FF48030094980394860012084F864
:10186000210000BF002084F8200000BF606B10B191
:101870002046616B8847284670BD0000800002400A
:10188000080402400146886B7047000070B50446AA
:10189000E06B05682068066894F8401004208840D2
:1018A0002840002875D006F004000028FAD02068EF
:1018B000006800F0200028B92068006820F00400CB
:1018C00021680860D5492068884254D9D3497839BD
:1018D0002068884201D1042049E0D0496439206859
:1018E000884201D1402042E0CC49503920688842EA
:1018F00001D100153BE0C9493C392068884202D13A
:101900004FF4804033E0C54928392068884202D12D
:101910004FF480202BE0C14914392068884202D15D
:101920004FF4800023E0BD492068884201D1C00403
:101930001DE0BB492068884201D1042017E0B84966
:1019400014312068884201D1402010E0B449283188
:101950002068884201D1001509E0B1493C31206876
:10196000884202D14FF4804001E04FF48020AC491E
:10197000091F086054E0A94978392068884201D1DC
:1019800004204AE0A54964392068884202D14020F9
:1019900043E04CE0A14950392068884201D100154C
:1019A0003BE09E493C392068884202D14FF4804098
:1019B00033E09A4928392068884202D14FF48020C8
:1019C0002BE0964914392068884202D14FF48000F8
:1019D00023E092492068884201D1C0041DE090496B
:1019E0002068884201D1042017E08D491431206815
:1019F000884201D1402010E089492831206888427E
:101A000001D1001509E086493C312068884202D1A5
:101A10004FF4804001E04FF48020804980394860D5
:101A2000E06A002802D02046E16A8847F4E094F892
:101A30004010022088402840002871D006F00200A3
:101A40000028FAD02068006800F0200040B9206823
:101A5000006820F00A0021680860012084F8210055
:101A60006E492068884254D96C4978392068884288
:101A700001D1022049E0694964392068884201D1D6
:101A8000202042E0654950392068884201D1401544
:101A90003BE062493C392068884202D14FF4005053
:101AA00033E05E4928392068884202D14FF4003083
:101AB0002BE05A4914392068884202D14FF40010B3
:101AC00023E056492068884201D180041DE0544932
:101AD0002068884201D1022017E051491431206862
:101AE000884201D1202010E04D49283120688842E9
:101AF00001D1401509E04A493C312068884202D1B1
:101B00004FF4005001E04FF400304549091F0860D0
:101B100054E0424978392068884202D102204AE0E4
:101B200057E03E4964392068884201D1202042E0D4
:101B30003A4950392068884201D140153BE0374985
:101B40003C392068884202D14FF4005033E03349D9
:101B500028392068884202D14FF400302BE02F4909
:101B600014392068884202D14FF4001023E02B4939
:101B70002068884201D180041DE0294920688842FC
:101B800001D1022017E0264914312068884201D192
:101B9000202010E0224928312068884201D14015D8
:101BA00009E01F493C312068884202D14FF40050BF
:101BB00001E04FF4003019498039486000BF00202F
:101BC00084F8200000BFA06A30B32046A16A88478D
:101BD00022E094F84010082088402840E0B106F048
:101BE0000800C8B12068006820F00E002168086075
:101BF00094F8401001208840E16B48600120A06308
:101C000084F8210000BF002084F8200000BF206B72
:101C100010B12046216B884770BD00008000024053
:101C2000080402400146002209B9012070471E4BFA
:101C3000086898420BD21D4B0868C01A1423B0FBE9
:101C4000F3F08000086419480838C8630AE0164BAE
:101C50000868C01A1423B0FBF3F08000086412482F
:101C60000838C863022081F821000868026843F63A
:101C7000F0708243D1E901031843CB6818430B6924
:101C800018434B6918438B691843CB6918430243C7
:101C90000868026000208863012081F8210000208C
:101CA00081F8200000BFC1E708040240080002409C
:101CB0002DE9F04104460D4616461F464FF0000838
:101CC00000BF94F82000012802D10220BDE8F08175
:101CD000012084F8200000BF94F8210001282CD1B5
:101CE000022084F821000020A0632068006820F012
:101CF0000100216808603B46324629462046FEF72F
:101D0000E7FEE06A30B12068006840F00E0021680C
:101D100008600BE02068006820F00400216808607B
:101D20002068006840F00A002168086020680068A8
:101D300040F001002168086006E000BF002084F840
:101D4000200000BF4FF002084046BFE770B50446D0
:101D500000F09AFA06462546681C10B1044800783F
:101D6000054400BF00F090FA801BA842FAD370BD72
:101D7000A80500202DE9F04104460E460127002564
:101D800000BF2648007E012802D10220BDE8F08174
:101D900001202249087600BF2068022813D14CF2A6
:101DA0005030FEF761FF90BB0120FEF7E3FE4CF2DE
:101DB0005030FEF759FF07461948006920F004002B
:101DC0001749086123E04CF25030FEF74DFFF0B99F
:101DD0004FF0FF303060A56812E02846FEF7DEFEC7
:101DE0004CF25030FEF740FF07460D48006920F0E6
:101DF00002000B4908610FB1356007E005F5006589
:101E0000D4E9021001EBC020A842E6D800BF00BF11
:101E100000200249087600BF3846B7E7C00F00200F
:101E2000002002400348006940F080000149086139
:101E300000207047002002402DE9FE4F05468B46EA
:101E400017469846012600240020029000BF24482F
:101E5000007E012802D10220BDE8FE8F012020492A
:101E6000087600BF4CF25030FEF7FEFE064686BBF9
:101E7000012D02D10120029006E0022D02D10220A4
:101E8000029001E00420029000241EE02201B946E5
:101E9000C24648465146FEF7B5F980B2019002208D
:101EA00000FB04B000900199FEF78CFE4CF250301C
:101EB000FEF7DAFE06460B48006920F001000949EA
:101EC000086106B104E0601CC4B202988442DDDB04
:101ED00000BF00BF00200249087600BF3046BBE7C4
:101EE000C00F00200020024000200849096901F0CD
:101EF000800151B10649054A5160064951601146B9
:101F0000096901F0800101B1012070470020024001
:101F100023016745AB89EFCD2DE9F8470246002341
:101F20009C467BE14FF0010808FA03F4D1F80080E9
:101F300008EA0400A0427DD1DFF8F4A2D1F80480C1
:101F4000A8EB0A09D0453AD014DCB8F1030F50D001
:101F500009DCB8F1000F31D0B8F1010F1CD0B8F195
:101F6000020F49D120E0B8F1110F18D0B8F1120FCB
:101F700042D11EE0B9F5881F25D006DCB9F5803FB7
:101F800020D0B9F5801F37D11AE0B9F5001F18D05D
:101F9000B9F5041F30D117E0D1F80CC02DE0D1F80D
:101FA0000C8008F1040C28E0D1F80C8008F1080C32
:101FB00023E0D1F80C8008F10C0C1EE000BF00BF3C
:101FC00000BF00BF00BF00BFD1F80880B8F1000F0C
:101FD00002D14FF0040C0BE0D1F80880B8F1010FEA
:101FE00003D14FF0080C146102E04FF0080C54616B
:101FF00003E04FF0000C00E000BF00BFFF2801D855
:10200000904601E002F104084646FF2802D84FEA54
:10201000830803E0A3F108084FEA88084746D6F88A
:1020200000804FF00F0909FA07F928EA09080CFAAD
:1020300007F900E07AE048EA0908C6F80080D1F81C
:10204000048008F08058B8F1805F6FD100BFDFF8DE
:10205000E481D8F8188048F00108DFF8D891C9F871
:102060001880C846D8F8188008F00108CDF800801C
:1020700000BF00BF4FEAB9384FEA930958F829501A
:102080004FEA83784FEA18794FF00F0808FA09F8F9
:1020900025EA0805DFF8A081424502D14FF000088B
:1020A00024E0DFF89881424502D14FF001081DE09D
:1020B000DFF88C81424502D14FF0020816E0DFF8CC
:1020C0008481424502D14FF003080FE0DFF87881A8
:1020D000424502D14FF0040808E0DFF87081424524
:1020E00002D14FF0050801E04FF006084FEA83796E
:1020F0004FEA197908FA09F848EA0505DFF850812E
:102100004FEA930948F82950D1F8048008F4801860
:10211000B8F5801F0BD1DFF83C81D8F8008048EA81
:102120000008DFF83091C9F800800AE075E0DFF8B8
:102130002481D8F8008028EA0008DFF81891C9F84F
:102140000080D1F8048008F40018B8F5001F0ED103
:10215000DFF8008108F10408D8F8008048EA000898
:10216000DFF8F09009F10409C9F800800DE0DFF80C
:10217000E48008F10408D8F8008028EA0008DFF8B5
:10218000D49009F10409C9F80080D1F8048008F45A
:102190000038B8F5003F0ED1DFF8B880A8F1040888
:1021A000D8F8008048EA0008DFF8A890A9F10409EF
:1021B000C9F800800DE0DFF89C80A8F10408D8F889
:1021C000008028EA0008DFF88C90A9F10409C9F81A
:1021D0000080D1F8048008F48038B8F5803F0ED133
:1021E000DFF87080A8F10808D8F8008048EA0008F5
:1021F000DFF86090A9F10809C9F800800DE0DFF868
:102200005480A8F10808D8F8008028EA0008DFF810
:102210004490A9F10809C9F800805B1CD1F800803E
:1022200028FA03F8B8F1000F7FF47CAEBDE8F88718
:10223000000011100010024000080140000C014095
:10224000001001400014014000180140001C014032
:102250000800014008040140024693680B400BB19E
:10226000012000E00020704710B5C26821EA020397
:1022700002EA010443EA0443036110BD0AB10161AB
:1022800001E00B04036170470148006870470000DB
:10229000A005002003480068034909780844014963
:1022A00008607047A0050020A805002010B5084868
:1022B000006840F0100006490860032000F0E2F8D2
:1022C0000F2000F007F800F05FF8002010BD0000BC
:1022D000002002402DE9F04188B004460027B846AE
:1022E000002600BF2348C06940F002002149C861B0
:1022F0000846C06900F00200019000BF00BF02A9BB
:1023000003A800F0DFFA069F1FB900F003FB0546A3
:1023100002E000F0FFFA45001748B5FBF0F0A0F12D
:10232000010816481649086040F2E7311448C160B8
:10233000C0F80480002101618160816100F0C4FD6A
:10234000064696B90E4800F013FE06466EB91D20EB
:1023500000F04AF8102C07D2002221461D2000F080
:1023600053F80848046000E00126304608B0BDE894
:10237000F08100000010024040420F0000040040C5
:10238000D4480020A405002008B500BF1448806987
:1023900040F00100124988610846806900F00100A0
:1023A000009000BF00BF00BF0846C06940F08050E9
:1023B000C8610846C06900F08050009000BF00BFAF
:1023C00000220F21901E00F01FF800BF0549486849
:1023D00020F0E06040F00070486000BF08BD0000E1
:1023E000001002400000014001460846002809DBB9
:1023F00000F01F0301229A4043099B0003F1E023F0
:10240000C3F8002100BF70472DE9F05F80460D46FC
:102410001646002703F056FE074639462A4633463D
:1024200001F00700C0F1070ABAF1040F02D94FF01A
:10243000040A01E0C0F1070AD14600F1040ABAF12A
:10244000070F02D24FF0000A01E0A0F1030AD446C0
:102450004FF0010A0AFA09FAAAF1010A0AEA020A85
:102460000AFA0CFA4FF0010B0BFA0CFBABF1010B63
:102470000BEA030B4AEA0B042146404603F02AFE0E
:10248000BDE8F09F00BF00F00702064B19684FF649
:10249000FF031940044B0B4343EA0221014B19602F
:1024A00000BF70470CED00E00000FA0500BF00BF60
:1024B00000BF00BF00BFBFF34F8F00BF00BF00BF12
:1024C0000948006800F4E06008490843001D064917
:1024D000086000BF00BF00BFBFF34F8F00BF00BF49
:1024E00000BF00BF00BFFDE70CED00E00000FA05F3
:1024F0002DE9F04706464FF000080025002700248C
:10250000A146042E37D004DC012E3CD0022E6CD123
:1025100060E0082E33D0102E67D13648446800683A
:1025200000F0807008B33448C4F38341475C04F47E
:10253000803078B12F484068C0F340402F4911F8EF
:10254000008004F4803040B12D48B0FBF8F000FB6F
:1025500007F502E02B4807FB00F52648406800F429
:102560008000B0F5800F01D1A94603E06800032187
:10257000B0FBF1F93AE000F0EDF9814636E000F009
:10258000E9F9814632E01B48046A04F44070B0F572
:10259000807F05D104F0020010B14FF4004918E02B
:1025A00004F44070B0F5007F07D11248406A00F093
:1025B000020010B149F640490BE004F44070B0F558
:1025C000407F06D10B48006800F4003008B14FF29C
:1025D00024490BE000F0AEF906494968C1F38131A6
:1025E000491C4900B0FBF1F900E000BF00BF4846BC
:1025F000BDE8F08700100240B67F0008C67F0008E3
:1026000000127A0000093D00F8B5044600260025B6
:10261000207800F0010000286BD000274348C069F3
:1026200000F0805070B900BF4048C06940F0805051
:102630003E49C8610846C06900F08050009000BF64
:1026400000BF01273A48006800F48070B0B93848EC
:10265000006840F4807036490860FFF715FE0646B2
:1026600006E0FFF711FE801B642801D90320F8BDA6
:102670002F48006800F480700028F2D02B48006AD0
:1026800000F440752DB3A08800F44070A84220D01B
:102690002648006A20F44075012026490860002081
:1026A00008602248056205F0010090B1FFF7ECFDDB
:1026B000064608E0FFF7E8FD801B41F288318842BA
:1026C00001D90320D3E71948006A00F0020000286E
:1026D000F0D01648006A20F440706168084313493E
:1026E0000862012F04D10846C06920F08050C861FB
:1026F00000BF207800F00200022807D10B48406894
:1027000020F44040A168084308494860207800F060
:102710001000102807D10548406820F48000616946
:102720000843024948600020A1E700000010024071
:10273000007000404004424270B504460D460CB99A
:10274000012070BD5A48006800F00700A8420ED270
:102750005748006820F0070028435549086008469C
:10276000006800F00700A84201D00120E9E72078C6
:1027700000F0020002281DD1207800F00400042897
:1027800005D14C48406840F4E0604A4948602078F0
:1027900000F00800082805D14648406840F4605021
:1027A000444948604348406820F0F000A16808436D
:1027B00040494860207800F0010078B36068012843
:1027C00006D13C48006800F4003090B90120B8E719
:1027D0006068022806D13748006800F0007040B9F0
:1027E0000120AEE73348006800F0020008B901207C
:1027F000A7E73048406820F00300616808432D498E
:102800004860FFF741FD064609E0FFF73DFD801BEC
:1028100041F28831884202D9032092E707E0254837
:10282000406800F00C006168B0EB810FEDD12048EA
:10283000006800F00700A8420ED91D48006820F08B
:10284000070028431A4908600846006800F007009E
:10285000A84201D0012074E7207800F00400042889
:1028600007D11448406820F4E060E168084311494A
:102870004860207800F00800082808D10D4840681A
:1028800020F46050216940EAC1000A49486000F024
:1028900061F808494968C1F30311074A515CC8400F
:1028A0000649086006480068FFF714FD002048E765
:1028B0000020024000100240C87F0008AC05002044
:1028C000A40500200F2202600D4A526802F00302A4
:1028D00042600B4A526802F0F0028260084A526875
:1028E00002F4E062C260064A526802F46052D20802
:1028F0000261044A126802F007020A607047000091
:1029000000100240002002400148006870470000AB
:10291000AC05002000B5FFF7F7FF04494968C1F393
:102920000221034A515CC84000BD00000010024073
:10293000D87F000800B5FFF7E7FF04494968C1F3F5
:10294000C221034A515CC84000BD00000010024093
:10295000D87F000870B50021002200240023002049
:10296000134D696801F00C05F5B1042D02D0082D56
:1029700019D101E00F4819E00F4DC1F38346AB5D5B
:1029800001F4803555B10A4D6D68C5F340450B4ED5
:10299000725D084D5D43B5FBF2F402E0084D03FBA8
:1029A00005F4204602E000BF024800BF00BF70BD32
:1029B0000010024000127A00A47F0008B47F0008D3
:1029C00000093D00F8B504460CB90120F8BD207897
:1029D00000F00100002878D0F848406800F00C00B2
:1029E00004280CD0F548406800F00C00082811D1EC
:1029F000F248406800F48030B0F5803F0AD1EF48DB
:102A0000006800F4003000285FD0606800285CD1C6
:102A10000120DBE700BF6068B0F5803F06D1E748E2
:102A2000006840F48030E549086028E0606858B9E3
:102A3000E248006820F48030E049086008460068F9
:102A400020F4802008601AE06068B0F5A02F0BD158
:102A5000DA48006840F48020D849086008460068D9
:102A600040F4803008600AE0D448006820F48030E8
:102A7000D24908600846006820F48020086000BF42
:102A8000606888B1FFF700FC054606E0FFF7FCFB35
:102A9000401B642801D9032098E7C848006800F467
:102AA00000300028F2D010E0FFF7EEFB054606E00C
:102AB000FFF7EAFB401B642801D9032086E7BF48E3
:102AC000006800F400300028F2D1207800F0020005
:102AD000022857D1B948406800F00C0050B1B748FF
:102AE000406800F00C00082818D1B448406800F491
:102AF000803098B9B148006800F0020020B1206928
:102B0000012801D0012061E7AC48006820F0F800FE
:102B1000616940EAC100A949086033E02069E8B171
:102B20000120A7490860FFF7AFFB054606E0FFF765
:102B3000ABFB401B022801D9032047E79F480068F0
:102B400000F002000028F2D09C48006820F0F80055
:102B5000616940EAC1009949086013E00020984982
:102B60000860FFF791FB054606E0FFF78DFB401B71
:102B7000022801D9032029E79048006800F00200EC
:102B80000028F2D1207800F0080008282DD1A06993
:102B9000B8B101208B490860FFF776FB054606E0D7
:102BA000FFF772FB401B022801D903200EE7834880
:102BB000406A00F002000028F2D0012002F00AFC76
:102BC00013E000207F490860FFF75EFB054606E042
:102BD000FFF75AFB401B022801D90320F6E677488D
:102BE000406A00F002000028F2D1207800F00400D2
:102BF000042873D100277148C06900F0805070B973
:102C000000BF6E48C06940F080506C49C8610846FA
:102C1000C06900F08050009000BF00BF01276A48E3
:102C2000006800F48070B0B96748006840F48070B4
:102C300065490860FFF728FB054606E0FFF724FB1F
:102C4000401B642801D90320C0E65F48006800F4F7
:102C500080700028F2D000BFE068012806D15748F4
:102C6000006A40F001005549086227E0E06858B961
:102C70005248006A20F00100504908620846006A84
:102C800020F00400086219E0E06805280BD14B48E9
:102C9000006A40F00400494908620846006A40F0B2
:102CA000010008620AE04548006A20F0010043493B
:102CB00008620846006A20F00400086200BFE0686D
:102CC000A0B1FFF7E1FA054609E0FFF7DDFA401B86
:102CD00041F28831884202D9032077E622E0374862
:102CE000006A00F002000028EFD012E0FFF7CCFAF3
:102CF000054608E0FFF7C8FA401B41F288318842D8
:102D000001D9032062E62D48006A00F00200002885
:102D1000F0D1012F05D12948C06920F08050274902
:102D2000C86100BFE069C8B32448406800F00C00E7
:102D3000082860D0E069022848D1002020490866B0
:102D4000FFF7A2FA054606E0FFF79EFA401B0228AD
:102D500001D903203AE61948006800F00070002805
:102D6000F2D1206AB0F5803F07D11448406820F4C2
:102D70000030A168084311494860D4E908010843BC
:102D80000E49496821F4741108430C494860012038
:102D90000B490866FFF778FA054607E03DE0FFF7C4
:102DA00073FA401B022801D903200FE6034800688C
:102DB00000F000700028F2D02FE000000010024068
:102DC000000042428004424200700040002014494A
:102DD0000866FFF759FA054606E0FFF755FA401B6B
:102DE000022801D90320F1E50E48006800F00070C8
:102DF0000028F2D111E0E069012800D1E6E5094898
:102E0000466806F48031206A814204D106F47011CC
:102E1000606A814201D00120D8E50020D6E500009B
:102E200000004242001002407047704730B5024631
:102E30000B4600BF92F83C00012801D1022030BDB2
:102E4000012082F83C0000BF022082F83D0010689B
:102E500044681068816824F070041868044310689E
:102E60004460144D1068A84213D0134D1068A84256
:102E70000FD01068B0F1804F0BD0104D1068A842F1
:102E800007D00F4D1068A84203D00E4D1068A8421D
:102E900005D121F08001586801431068816001204C
:102EA00082F83D0000BF002082F83C0000BF00BF58
:102EB000C5E70000002C0140003401400004004040
:102EC00000080040000C004010B504460CB9012079
:102ED00010BD94F83D0028B9002084F83C0020463D
:102EE00000F026F8022084F83D00211D206802F041
:102EF0007DFC012084F8460000BF84F83E000121DB
:102F00003F200155402001554120015500BF00BF21
:102F1000012084F8420043200155442001554520FA
:102F2000015500BF012084F83D000020D0E70000DB
:102F300038B504462068B0F1804F15D100BF0B486A
:102F4000C06940F001000949C8610846C06900F045
:102F50000100009000BF00BF002205211C20FFF7E8
:102F600053FA1C20FFF740FA38BD00000010024061
:102F7000014691F83D00012801D001207047022050
:102F800081F83D000868C06840F001000B68D86017
:102F9000164B0868984213D0154B086898420FD01A
:102FA0000868B0F1804F0BD0124B0868984207D0E8
:102FB000114B0868984203D0104B086898420CD116
:102FC0000868806800F00702062A0CD008680068CC
:102FD00040F001000B68186005E00868006840F0E8
:102FE00001000B6818600020C8E70000002C0140B9
:102FF000003401400004004000080040000C004084
:103000002DE9F04104460D46002700BF94F83C002E
:10301000012802D10220BDE8F081012084F83C00A3
:1030200000BF022084F83D002068866826F07706FD
:1030300026F47F46206886602868502833D00CDC50
:10304000202850D004DC00284BD0102851D149E072
:10305000302849D040284CD139E060282DD0702844
:1030600007D0B0F5805F03D0B0F5005F41D10DE02F
:1030700041E0D5E902136A68206802F005FC206887
:10308000866846F077062068866034E0D5E902134A
:103090006A68206802F0F8FB2068806840F480408D
:1030A0002168886027E0EA686968206802F000FC0F
:1030B0005021206802F0F3FB1DE0EA68696820688F
:1030C00002F009FC6021206802F0E9FB13E0EA68E5
:1030D0006968206802F0ECFB4021206802F0DFFB09
:1030E00009E000BF00BF00BF2968206802F0D7FBDD
:1030F00001E0012700BF00BF012084F83D0000BFB0
:10310000002084F83C0000BF384684E7704710B5C3
:10311000044620680069C0F34000D8B12068C06848
:10312000C0F34000B0B16FF00200216808610120D7
:1031300020772068806900F0030018B12046FFF76F
:10314000E5FF05E0204600F0ADF8204600F0ABF8C2
:103150000020207720680069C0F38000D8B1206883
:10316000C068C0F38000B0B16FF00400216808614E
:10317000022020772068806900F4407018B1204652
:10318000FFF7C4FF05E0204600F08CF8204600F071
:103190008AF80020207720680069C0F3C000D8B109
:1031A0002068C068C0F3C000B0B16FF008002168AB
:1031B0000861042020772068C06900F0030018B17E
:1031C0002046FFF7A3FF05E0204600F06BF82046FD
:1031D00000F069F80020207720680069C0F3001033
:1031E000D8B12068C068C0F30010B0B16FF0100013
:1031F00021680861082020772068C06900F44070C9
:1032000018B12046FFF782FF05E0204600F04AF89B
:10321000204600F048F8002020772068006900F080
:10322000010058B12068C06800F0010030B16FF0B3
:10323000010021680861204600F036F82068006926
:10324000C0F3C01058B12068C068C0F3C01030B1DE
:103250006FF08000216808612046FFF7E5FD2068D7
:103260000069C0F3801058B12068C068C0F38010B6
:1032700030B16FF0400021680861204600F020F86E
:1032800020680069C0F3401058B12068C068C0F3DE
:10329000401030B16FF02000216808612046FFF730
:1032A000C4FD10BD7047704710B50446034920683F
:1032B000884201D1FEF7EEFF10BD0000000400407F
:1032C0007047704710B5044600BF00BF21680C313D
:1032D00051E8001F21F4907021680C3141E8000290
:1032E000002AF3D100BF00BF00BF2168143151E8AC
:1032F000001F21F001002168143141E80002002A7A
:10330000F3D100BF206B01280ED100BF00BF2168A0
:103310000C3151E8001F21F0100021680C3141E808
:103320000002002AF3D100BF2068406900F040008D
:1033300000B300BF00BF2168143151E8001F21F025
:1033400040002168143141E80002002AF3D100BF97
:10335000E06B78B10020E16B4863E06BFEF792F917
:1033600040B1E06BFEF78EFA202803D11020606494
:10337000032010BD0020E085202084F842000020BA
:10338000206300BFF5E770B504460025206840695A
:10339000C0F3C01594F84100212817D1B5B100BF82
:1033A00000BF2168143151E8001F21F0800021681E
:1033B000143141E80002002AF3D100BFA06B10B124
:1033C000A06BFEF75FF9204602F07DFB20684069A4
:1033D000C0F3801594F84200222817D1B5B100BF80
:1033E00000BF2168143151E8001F21F0400021681E
:1033F000143141E80002002AF3D100BFE06B10B1A4
:10340000E06BFEF73FF9204602F017FB002070BD8D
:10341000704700002DE9F84F0446206805682068D1
:10342000C668206847694FF00009CA4605F00F09D1
:10343000B9F1000F0AD105F0200038B106F02000E4
:1034400020B1204602F052FBBDE8F88FB9F1000F21
:103450007BD007F0010018B906F49070002874D0F2
:1034600005F0010030B106F4807018B1606C40F0D6
:103470000100606405F0040030B107F0010018B1EC
:10348000606C40F00200606405F0020030B107F0AB
:10349000010018B1606C40F00400606405F00800A1
:1034A00048B106F0200010B907F0010018B1606CB7
:1034B00040F008006064606C002845D005F02000F2
:1034C00028B106F0200010B1204602F00FFB206862
:1034D0004069C0F3801A606C00F0080010B9BAF1BE
:1034E000000F2CD0204602F0A8FA2068406900F0B6
:1034F000400000B300BF00BF2168143151E8001F35
:1035000021F040002168143141E80002002AF3D183
:1035100000BFE06B50B17748E16B4863E06BFEF7AA
:10352000DDF888B1E06B416B88470DE02046FFF77E
:103530006FFF09E009E02046FFF76AFF04E020463C
:10354000FFF766FF002060647EE7206B012877D1DB
:1035500005F01000002873D006F010000028FAD003
:1035600000BF00200090206800680090206840683C
:10357000009000BF00BF2068406900F040000028B4
:103580005FD0E06B006840681FFA80F8B8F1000F68
:1035900055D0A08D404552DDA4F82E80E06B8069A7
:1035A000202843D000BF00BF21680C3151E8001F24
:1035B00021F4807021680C3141E80002002AF3D127
:1035C00000BF00BF00BF2168143151E8001F21F087
:1035D00001002168143141E80002002AF3D100BF44
:1035E00000BF00BF2168143151E8001F21F04000E6
:1035F0002168143141E80002002AF3D100BF2020E5
:1036000084F842000020206300BF00BF21680C3115
:1036100051E8001F21F0100021680C3141E8000240
:10362000002AF3D100BFE06BFEF72CF802206063A4
:10363000A08DE28D801A81B22046FFF742FE03E79B
:1036400042E0A08DE18D401A1FFA80F8E08DD0B3E2
:10365000B8F1000F37D000BF00BF21680C3151E82E
:10366000001F21F4907021680C3141E80002002A0B
:10367000F3D100BF00BF00BF2168143151E8001F23
:1036800021F001002168143141E80002002AF3D141
:1036900000BF202084F842000020206300BF00BF4C
:1036A00021680C3151E8001F21F0100021680C3115
:1036B00041E80002002AF3D100BF022060634146C6
:1036C0002046FFF7FEFDBFE605F0800030B106F0B2
:1036D000800018B1204602F069FBB5E605F0400015
:1036E00030B106F0400018B1204602F0DCF9ABE63C
:1036F00000BFA9E6FF58000810B504460CB9012028
:1037000010BDA06900B100E000BF94F8410028B9E5
:10371000002084F84000204600F02AF8242084F895
:1037200041002068C06820F400502168C86020462D
:1037300002F05AFA2068006920F49040216808617C
:103740002068406920F02A00216848612068C0682C
:1037500040F400502168C86000206064202084F894
:10376000410084F842000020606300BFC8E7000009
:1037700010B586B004460020029003900490059096
:103780006249206888426AD100BF6148806940F47C
:1037900080405F4988610846806900F4804001905C
:1037A00000BF00BF00BF0846806940F00400886188
:1037B0000846806900F00400019000BF00BF481572
:1037C0000290022003900320059002A95148FEF7C1
:1037D000A3FB4FF48060029000200390049002A9A4
:1037E0004C48FEF799FB4C484C4908600020486063
:1037F00000214A4881608021C1600021016141614E
:103800008161C161FEF70EFA08B1FDF7B0F900BFA2
:103810004248E063446200BF3F48143840490860B2
:103820001020486000213E4881608021C160002155
:10383000016141618161C161FEF7F4F908B1FDF7F1
:1038400096F900BF3648A063446200BF00220521FC
:103850002520FEF7D9FD2520FEF7C6FD54E03149AD
:103860002068884250D100BF2948C06940F48020B8
:103870002749C8610846C06900F48020019000BF54
:1038800000BF00BF0846806940F008008861084614
:10389000806900F00800019000BF00BF0815029089
:1038A000022003900320059002A91F48FEF734FB75
:1038B0004FF40060029000200390049002A91A487F
:1038C000FEF72AFB14482838184908600020486091
:1038D0000021164881608021C160002101614161A1
:1038E0008161C161FEF79EF908B1FDF740F900BFA3
:1038F0000E48E063446200BF002205212720FEF746
:1039000083FD2720FEF770FD06B010BD0038014092
:103910000010024000080140580002400848002002
:103920004C48002000480040000C01409048002016
:1039300070B504460D46164694F8420020280BD177
:1039400005B10EB9012070BD002020633246294622
:10395000204602F0C7F9F6E70220F4E76FF02001F5
:1039600002681160891002681160704770472DE984
:10397000F84F04460E46174699464FF0000A94F851
:10398000410020284AD106B117B90120BDE8F88FBF
:1039900000206064212084F84100FEF775FC824617
:1039A000A784E784A068B0F5805F04D1206910B9CE
:1039B0000025B04602E035464FF000081BE05346B4
:1039C000002280212046CDF8009002F01FFA08B1B5
:1039D0000320DBE745B9B8F80000C0F30800216810
:1039E000486008F1020803E02878216848606D1CEF
:1039F000E08C401EE084E08C0028E0D15346002299
:103A000040212046CDF8009002F000FA08B10320D2
:103A1000BCE7202084F841000020B7E70220B5E78A
:103A200010B5034693F84100202813D101B10AB91B
:103A3000012010BD19629A84DA8400205864212084
:103A400083F841001868C06840F080001C68E0609E
:103A50000020EEE70220ECE76FF020010268116021
:103A6000891002681160704700BFFEE72DE9FC4134
:103A700006460C46082204F110016846FDF758F886
:103A8000208AC0F3C505382D02D2C5F1380001E007
:103A9000C5F1780007463A460A49204600F014FC72
:103AA00008226946204600F00FFC102221463046CD
:103AB000FDF73EF858220021204600F051FCBDE8F9
:103AC000FC8100006005002000224261026105497E
:103AD0000160054941600349C94381600249C94306
:103AE000C16070470123456789ABCDEF2DE9F043F5
:103AF00091B080468946D8F80040D8F80450D8F8EC
:103B00000860D8F80C704022494601A8FCF7F7FF7E
:103B100005EA060027EA0501084301990844FE4921
:103B200008440444E00140EA54642C4404EA0500DB
:103B300026EA0401084302990844F8490844074466
:103B4000380340EA1757274407EA040025EA07012B
:103B5000084303990844F24908440644700440EAC3
:103B6000D6363E4406EA070024EA060108430499D3
:103B70000844EC4908440544A80540EA9525354425
:103B800005EA060027EA0501084305990844E649C5
:103B900008440444E00140EA54642C4404EA05006B
:103BA00026EA0401084306990844E049084407440A
:103BB000380340EA1757274407EA040025EA0701BB
:103BC000084307990844DA4908440644700440EA67
:103BD000D6363E4406EA070024EA0601084308995F
:103BE0000844D44908440544A80540EA95253544CD
:103BF00005EA060027EA0501084309990844CE4969
:103C000008440444E00140EA54642C4404EA0500FA
:103C100026EA040108430A990844C84908440744AD
:103C2000380340EA1757274407EA040025EA07014A
:103C300008430B990844A0F524404F38064470040B
:103C400040EAD6363E4406EA070024EA0601084365
:103C50000C990844BA4908440544A80540EA95254A
:103C6000354405EA060027EA050108430D99084492
:103C7000B44908440444E00140EA54642C4404EA92
:103C8000050026EA040108430E990844AE49084499
:103C90000744380340EA1757274407EA040025EA97
:103CA000070108430F990844A849084406447004D2
:103CB00040EAD6363E4406EA070024EA06010843F5
:103CC00010990844A24908440544A80540EA9525EE
:103CD000354405EA070026EA07010843029908442B
:103CE0009C4908440444600140EAD4642C4404EA3A
:103CF000060025EA06010843079908449649084446
:103D00000744780240EAD757274407EA050024EA27
:103D1000050108430C990844904908440644B0033F
:103D200040EA96463E4406EA040027EA04010843B6
:103D3000019908448A4908440544280540EA153594
:103D4000354405EA070026EA0701084306990844B6
:103D5000844908440444600140EAD4642C4404EAE1
:103D6000060025EA060108430B9908447E490844E9
:103D70000744780240EAD757274407EA050024EAB7
:103D80000501084310990844784908440644B003E3
:103D900040EA96463E4406EA040027EA0401084346
:103DA00005990844724908440544280540EA153538
:103DB000354405EA070026EA070108430A99084442
:103DC0006C4908440444600140EAD4642C4404EA89
:103DD000060025EA060108430F990844664908448D
:103DE0000744780240EAD757274407EA050024EA47
:103DF0000501084304990844604908440644B00397
:103E000040EA96463E4406EA040027EA04010843D5
:103E1000099908445A4908440544280540EA1535DB
:103E2000354405EA070026EA070108430E990844CD
:103E3000544908440444600140EAD4642C4404EA30
:103E4000060025EA06010843039908444E49084440
:103E50000744780240EAD757274407EA050024EAD6
:103E60000501084308990844484908440644B0033A
:103E700040EA96463E4406EA040027EA0401084365
:103E80000D990844424908440544280540EA15357F
:103E9000354485EA06007840069908443D490844BF
:103EA0000444200140EA14742C4484EA0500704064
:103EB00009990844384908440744F80240EA57572A
:103EC000274487EA040068400C99084433490844B1
:103ED0000644300440EA16463E4486EA0700604045
:103EE0000F9908442E4908440544E80540EA552541
:103EF000354485EA06007840029908442949084477
:103F00000444200140EA14742C4484EA0500704003
:103F100005990844244949E078A46AD756B7C7E808
:103F2000DB702024EECEBDC1AF0F7CF52AC68747DB
:103F3000134630A8019546FDD8988069AFF7448BA9
:103F4000BED75C892211906B937198FD8E4379A640
:103F50002108B44962251EF640B340C0515A5E267E
:103F6000AAC7B6E95D102FD65314440281E6A1D842
:103F7000C8FBD3E7E6CDE121D60737C3870DD5F4DB
:103F8000ED145A4505E9E3A9F8A3EFFCD9026F67E0
:103F90008A4C2A8D4239FAFF81F6718722619D6D24
:103FA0000C38E5FD44EABEA4A9CFDE4B0844074423
:103FB000F80240EA5757274487EA04006840089906
:103FC0000844A74908440644300440EA16463E44E3
:103FD00086EA070060400B990844A249084405445A
:103FE000E80540EA5525354485EA060078400E99F3
:103FF00008449D4908440444200140EA14742C44B8
:1040000084EA05007040019908449849084407442F
:10401000F80240EA5757274487EA040068400499A9
:104020000844934908440644300440EA16463E4496
:1040300086EA07006040079908448E490844054411
:10404000E80540EA5525354485EA060078400A9996
:104050000844894908440444200140EA14742C446B
:1040600084EA050070400D990844844908440744D7
:10407000F80240EA5757274487EA0400684010993D
:1040800008447F4908440644300440EA16463E444A
:1040900086EA07006040039908447A4908440544C9
:1040A000E80540EA5525354465EA07007040019966
:1040B0000844754908440444A00140EA94642C442F
:1040C00064EA0600684008990844704908440744B7
:1040D000B80240EA9757274467EA050060400F9905
:1040E00008446B4908440644F00340EA56463E44FF
:1040F00066EA040078400699084466490844054485
:10410000680540EAD525354465EA070070400D99F9
:104110000844614908440444A00140EA94642C44E2
:1041200064EA06006840049908445C49084407446E
:10413000B80240EA9757274467EA050060400B99A8
:104140000844574908440644F00340EA56463E44B2
:1041500066EA04007840029908445249084405443C
:10416000680540EAD525354465EA0700704009999D
:1041700008444D4908440444A00140EA94642C4496
:1041800064EA060068401099084448490844074416
:10419000B80240EA9757274467EA0500604007994C
:1041A0000844434908440644F00340EA56463E4466
:1041B00066EA040078400E9908443E4908440544E4
:1041C000680540EAD525354465EA07007040059941
:1041D0000844394908440444A00140EA94642C444A
:1041E00064EA060068400C990844344908440744CE
:1041F000B80240EA9757274467EA050060400399F0
:1042000008442F4908440644F00340EA56463E4419
:1042100066EA040078400A9908442A49084405449B
:10422000680540EAD5253544D8F800002044C8F890
:104230000000D8F804002844C8F80400D8F80800A2
:104240003044C8F80800D8F80C003844C8F80C000E
:104250004022002101A800F083F811B0BDE8F083EE
:10426000604BBBF670BCBFBEC67E9B28FA27A1EA96
:104270008530EFD4051D880439D0D4D9E599DBE623
:10428000F87CA21F6556ACC4442229F497FF2A4348
:10429000A72394AB39A093FCC3595B6592CC0C8FD8
:1042A0007DF4EFFFD15D84854F7EA86FE0E62CFEA4
:1042B000144301A3A111084E827E53F735F23ABD93
:1042C000BBD2D72A91D386EB2DE9F0470446884626
:1042D0001546208AC0F3C509206900EBC50020619E
:1042E000B0EBC50F02D26069401C6061606900EBF1
:1042F00055716161C9F14007BD421BD304F118013A
:1043000001EB09003A46414600F020F804F118019B
:104310002046FFF7EBFB3E4605E008EB0601204692
:10432000FFF7E4FB403606F13F00A842F5D34FF01B
:10433000000900E00026AA1B08EB060104F118039F
:1043400003EB090000F002F8BDE8F08710B5034662
:10435000002002E00C5C1C54401C9042FAD310BDBB
:1043600010B50346002001E01954401C9042FBD3D5
:1043700010BD00000EB500200090019002901E4874
:104380001E49086081151D488160002101730121CB
:10439000017581614FF46021C161002017494860B7
:1043A000032116480161FCF703FF08B1FCF7DFFBAE
:1043B0000A200090012001900720029069460F48D2
:1043C000FCF7B8FD08B1FCF7D2FB0B2000900220EF
:1043D000019069460948FCF7ADFD08B1FCF7C7FB41
:1043E0000C2000900320019069460448FCF7A2FDD0
:1043F00008B1FCF7BCFB0EBD00240140540F0020A7
:1044000008B500BF1248406940F0010010494861FA
:104410000846406900F00100009000BF00BF002284
:1044200005210D20FDF7F0FF0D20FDF7DDFF002237
:1044300005210E20FDF7E8FF0E20FDF7D5FF002235
:1044400005210F20FDF7E0FF0F20FDF7CDFF08BD90
:104450000010024000B59DB01C22184916A8FBF7B9
:10446000E1FE002116A802F040FB154908601C225D
:1044700012491C310FA8FBF7D5FE00210FA802F04E
:1044800034FB104908601C220C49383108A8FBF79E
:10449000C9FE002108A802F028FB0B4908601C2275
:1044A0000649543101A8FBF7BDFE002101A802F026
:1044B0001CFB064908601DB000BD0000347F0008E9
:1044C00064000020680000206C00002070000020C4
:1044D00000B585B00020019002900390049000BFC9
:1044E0003A48806940F01000384988610846806980
:1044F00000F01000009000BF00BF00BF08468069B8
:1045000040F0200088610846806900F0200000909B
:1045100000BF00BF00BF0846806940F0040088610A
:104520000846806900F00400009000BF00BF00BF93
:104530000846806940F0080088610846806900F0FC
:104540000800009000BF00BF002241F2790120481E
:10455000FDF794FE4FF6F87001900320029001A938
:104560001C48FDF7D9FCFF20019000200290039029
:1045700001A91948FDF7D0FC41F279000190012012
:104580000290002003900220049001A91048FDF73A
:10459000C3FC4EF2863001900320029001A90C4822
:1045A000FDF7BAFC4FF4194001900320029001A9D5
:1045B0000948FDF7B1FC042001900320029001A9F5
:1045C0000648FDF7A9FC05B000BD00000010024040
:1045D000000C01400010014000080140001401409F
:1045E00000B587B0002003900490059006900190DC
:1045F00002904FF080401549086040F21F3048603B
:1046000000211248816041F63F71C16000210161C3
:1046100080218161FEF758FC08B1FCF7A8FA4FF43D
:104620008050039003A90948FEF7EAFC08B1FCF7A3
:104630009EFA00200190029001A90448FEF7F6FBC3
:1046400008B1FCF794FA07B000BD000084320020E6
:1046500010B50B480B4908604FF416504860002114
:1046600008488160C16001610C21416100218161C4
:10467000C161FFF741F808B1FCF779FA10BD0000FD
:10468000003801407847002010B50B480B490860FE
:104690004FF416504860002108488160C1600161F4
:1046A0000C21416100218161C161FFF725F808B14A
:1046B000FCF75DFA10BD000000480040C047002034
:1046C00000BFFEE710B586B0FE480078012831D162
:1046D0000621FD4801F0C8FEFB498979FA4AD279E2
:1046E00041EA02218842F2D1F84800880A2821DAFA
:1046F000F5480078F649097888421CD1F24840789C
:10470000032818D1F0488078A8B9EF48C07801286C
:1047100011D1ED48007970B9EB48407901280AD1F0
:1047200007200090EB48037802220321E848008824
:1047300002F02CFE91E3E4480078E54909788842CC
:104740001CD1E1484078032818D1DF488078A8B907
:10475000DD48C078022811D1DB48007970B9DA4809
:10476000407901280AD107200090DB480378022213
:104770000321D748008802F009FE6EE3D248007892
:10478000D349097888421CD1CF484078032818D1F2
:10479000CD488078A8B9CC48C078032811D1CA4840
:1047A000007970B9C848407901280AD107200090E3
:1047B000CA48038802220321C548008802F0E6FDAA
:1047C0004BE3C1480078C249097888421CD1BE48F1
:1047D0004078032818D1BC488078A8B9BA48C07876
:1047E000042811D1B848007970B9B7484079012838
:1047F0000AD107200090BA48038802220321B44856
:10480000008802F0C3FD28E3AF480078B04909787A
:1048100088421CD1AC484078032818D1AA48807837
:10482000A8B9A948C078052811D1A748007970B95E
:10483000A548407901280AD107200090A94803889B
:1048400002220321A248008802F0A0FD05E39E4851
:1048500000789F49097888421FD19B4840780328F7
:104860001BD199488078C0B99748C078012814D1E5
:104870009548007988B99448407902280DD10920DB
:1048800095490978CDE90010924803780422032164
:104890008F48008802F0E4FDDFE28B4800788C4905
:1048A0000978884222D18848407803281ED186485A
:1048B0008078D8B98448C078012817D18248007917
:1048C000A0B981484079032810D10B218348008882
:1048D000814A1278CDE9002002917E4803780622B1
:1048E00003217B48008802F059FCB6E27648007844
:1048F00077490978884225D173484078032821D127
:1049000071488078F0B97048C07801281AD16E4893
:104910000079B8B96C484079042813D10D22704849
:1049200000886E4909886C4B1B78CDE90031CDE9D0
:10493000020268480378082203216548008802F0D3
:1049400075FC8AE26048007861490978884228D17C
:104950005D484078032824D15B48807808BB5A48DA
:10496000C07801281DD158480079D0B956484079FF
:10497000052816D10F215B48028859480088574BFB
:104980001B88CDE90130CDE9032153480078009020
:10499000504803780A2203214D48008802F09AFC0F
:1049A0005BE2494800784A49097888421FD1464865
:1049B000407803281BD144488078C0B94248C07869
:1049C000022814D14048007988B93F48407902282C
:1049D0000DD1092041490988CDE900103E480378EE
:1049E000042203213A48008802F03AFD35E23648B5
:1049F000007837490978884222D133484078032823
:104A00001ED131488078D8B92F48C078022817D1F4
:104A10002D480079A0B92C484079032810D10B21EA
:104A20002F4800882D4A1288CDE9002002912A489B
:104A30000378062203212648008802F0AFFB0CE22F
:104A40002148007822490978884225D11E484078BB
:104A5000032821D11C488078F0B91B48C07802286F
:104A60001AD119480079B8B917484079042813D1E8
:104A70000D211C4800881A4A1288184B1B88CDE962
:104A80000032CDE9020114480378082203211048BE
:104A9000008802F0CBFBE0E10B4800780C49097874
:104AA000884232D10848407803282ED106488078C1
:104AB00058BB0548C078032827D10348007920BB9C
:104AC000014811E025050020CC3A002026050020F1
:104AD0005200002060000020610000207A000020C9
:104AE0007C00002078000020407902280DD10920A8
:104AF000DB490988CDE90010DA4803880422032144
:104B0000D948008802F0ACFCA7E1D8480078D64923
:104B10000978884222D1D548407803281ED1D3484D
:104B20008078D8B9D148C078032817D1CF48007908
:104B3000A0B9CE484079032810D10B21CC48008879
:104B4000C74A1288CDE900200291C6480388062290
:104B50000321C548008802F021FB7EE1C3480078AC
:104B6000C149097888421FD1C048407803281BD129
:104B7000BE488078C0B9BD48C078042814D1BB486D
:104B8000007988B9B948407902280DD10920B8497F
:104B90000988CDE90010B248038804220321B248F5
:104BA000008802F05DFC58E1B0480078FA281BD17B
:104BB000AE484078032817D1AC488078A0B9AB48FC
:104BC000C078AA2810D1A948007968B9A7484079C7
:104BD000012809D107200090A3480388022203215D
:104BE000FA2002F0D3FB38E1A04800789E4909780A
:104BF000884224D19D484078032820D19B48807862
:104C000050281CD19948C078C8B998480079B0B9E3
:104C100096484079022812D109219648008880B22E
:104C2000CDE90001934800684FF6FF7101EA104397
:104C3000042203218C48008802F012FC0DE18B480D
:104C4000007889490978884229D18848407806281F
:104C500025D18648807810BB8448C07802281ED1B0
:104C600082480079D8B98149487902F073FC05225D
:104C70007E49814801F068F97C4840797B4C247971
:104C800040EA04237948C078784CA47840EA0422AA
:104C9000764841787448008802F0AEFBDDE0734846
:104CA000007871490978884229D1704840780628EF
:104CB00025D16E48807810BB6C48C0780A281ED178
:104CC0006A480079D8B969484079012817D100228B
:104CD00066496A4801F038F964484079634C2479A0
:104CE00040EA04236148C078604CA47840EA04227A
:104CF0005E4841785C48008802F07EFBADE05B488E
:104D0000007859490978884229D1584840780628BE
:104D100025D15648807810BB5448C0780B281ED146
:104D200052480079D8B951484079012817D100225A
:104D30004E49534801F008F94C4840794B4C2479CE
:104D400040EA04234948C078484CA47840EA042249
:104D5000464841784448008802F04EFB7DE04348D5
:104D6000007841490978884229D14048407806288E
:104D700025D13E48807810BB3C48C0780C281ED115
:104D80003A480079D8B93949487902F019FC052226
:104D900036493C4801F0D8F834484079334C2479FE
:104DA00040EA04233148C078304CA47840EA042219
:104DB0002E4841782C48008802F01EFB4DE02B481D
:104DC000007829490978884225D128484078062862
:104DD00021D126488078F0B92448C078AA281AD171
:104DE00022480079B8B905222049274801F0ACF8DB
:104DF0001E4840791D4C247940EA04231B48C078A2
:104E00001A4CA47840EA04221848417816480088D1
:104E100002F0F2FA21E01548007813490978884237
:104E200017D112484078062813D11048807880B9ED
:104E30000E48C078CC280CD10C480079A52808D1A0
:104E40000A4840795A2804D101F046FBFDF72EFBB1
:104E500003E001F041FB02F063F906B010BD000071
:104E60007C0000207A00002052000020CC3A002074
:104E700078000020580000200008070800180708E4
:104E800000200708001007080000070800BFFEE721
:104E9000FEB50020F9490870F948407AF849097AC6
:104EA00040EA0120F7490880F7480588F7A103C9BF
:104EB000CDE90101F248C079F64908704FF48061EC
:104EC000F548FBF7C8F94FF48061F448FBF7C3F9E4
:104ED000F0480078012804D002287DD004287CD135
:104EE000ADE12822E6490A31ED48FBF79BF9802124
:104EF000E3480A3001F028FBEA490880E81EE0494F
:104F0000095C281FDE4A105C41EA0020E64908805F
:104F1000E4480088098888427ED100240AE0E348FA
:104F20002044017904F10A00D54A105C814200D086
:104F300002E0641C582CF2DB00BF322C6DDA002436
:104F40000FE00A2000EB4400CD49085C0B2101EB87
:104F50004401CB4A515C40EA0120CF4921F81400BA
:104F6000641C192CEDDB1922D049091DCA48FBF736
:104F7000C9FE322001F009FB0120CD490860CB4970
:104F80001B31CC4802F0DCF8C948006830B3C9488E
:104F9000007800F00F0042F210714843C54949788B
:104FA00001F00F0101EB4102C2EBC11100EBC101A5
:104FB000C048807800F00F0000EBC00202EB001048
:104FC00001EB8000BB49C97801F00F0101EB8101C1
:104FD00000EB4100B74902E0BBE0DFE106E0097900
:104FE00001F00F010844B449086022E0B14800789C
:104FF00000F00F004FF47A714843AE49497801F050
:105000000F0101EBC10202EB011100EB8100A94984
:10501000897801F00F0101E081E061E001EB81019D
:1050200000EB4101A348C07800F00F000844A249FA
:105030000860A1480068A1490860A14801F0AEFAE3
:10504000FCF752FF9D4800239D4902680120FCF7B0
:10505000F3FEFCF7E7FE96480068F8B1102293498A
:1050600021319848FBF738FE082297499548FBF70D
:1050700049FE00200FE0934931F810104FF47F42B1
:1050800002EA01218F4A32F8102041EA12218D4AAA
:1050900022F81010401C0828EDDB1EE01022834986
:1050A00020318848FBF718FE082287498548FBF71E
:1050B00029FE00200FE0834931F810104FF47F42A1
:1050C00002EA01217F4A32F8102041EA12217D4A8A
:1050D00022F81010401C0828EDDB7C487C49086051
:1050E0004FF480616648FBF7B6F8502001F04DFAA6
:1050F00078488079009077484079764E367940EA52
:1051000006237448C078734EB67840EA0622714888
:1051100041787148008802F0E3F900BF0EE04FF4D7
:1051200080615748FBF797F801A8FBF79FF886B214
:105130006423324601A96948FEF719FC4FF48061E7
:105140005548FBF788F84FF480615448FBF783F823
:1051500025E180214A480A3001F0F6F951490880DA
:10516000E81E4749095C281F454A105C01EB0020F6
:105170004D4908804B480088098888425ED1002448
:105180000FE00A2000EB44003D49085C0B2101EBD5
:1051900044013B4A515C40EA01203F4921F8140098
:1051A000641C402CEDDB4022494801683A48FBF77B
:1051B000A9FD474800688030454908600122114632
:1051C0004748FDF75BF80120FCF7C0FD00220121F4
:1051D0004348FDF753F82A48C0782949897840EABE
:1051E00001203B49098889B288420AD001A8FBF70F
:1051F0003DF886B26423324601A93848FEF7B7FB72
:10520000CDE04FF480611E48FBF725F8502001F0F7
:10521000BCF93048807900902E4840792D4E36797F
:1052200040EA06232B48C0782A4EB67840EA062288
:10523000284841782848008802F052F9AFE08021E0
:105240000F480A3001F080F916490880E81E0C4921
:10525000095C281F0A4A105C01EB002012490880F3
:1052600010480088098888426FD108220F490E3102
:105270001C48FBF731FD002046E00000240500201B
:10528000CC32002016000020260500206572726FC7
:10529000720D0A00040000208A0600208A0A0020FD
:1052A000180600201C0000201E0000207AF00708CD
:1052B0003000002060060020240000203400002080
:1052C000004807087A06002000500708000004087C
:1052D00020000020CC3A0020520000207847002017
:1052E000000C0140060000202E4931F810104FF448
:1052F0007F4202EA01212B4A32F8102041EA1221B2
:10530000284A22F81010401C0428EDDB26492548C5
:1053100001F0FCF8254801F041F9FCF7E5FD2248D1
:105320000023224902680220FCF786FDFCF77AFD83
:105330001F4801681F48FBF70BFB1F490860084620
:10534000006818B100F080F827E016E01BA11F48A4
:1053500000F0A4FE0646502001F017F9B2B21B4936
:105360001B48FEF75DFB02E00120FCF7EFFC18484C
:1053700090F841002128F7D00FE0502001F005F906
:1053800001A8FAF773FF86B26423324601A91048D8
:10539000FEF7EDFA502001F0F8F800E000BF00BF82
:1053A000FEBD000006000020580000200040070855
:1053B00034000020000004082C00002063686563AE
:1053C0006B3D6572726F720D0A000000CC320020D6
:1053D0007847002008B508490968C9084FF47A726F
:1053E000B1FBF2F14143009100BF00BF00994A1E9A
:1053F00000920029F9D108BDAC05002070B5044623
:105400000D4629462046FCF727FF08B9012070BD4C
:105410000020FCE708B509480949086008460088EB
:1054200080B2ADF8020008460068000CADF800003C
:10543000022204496846FBF765FC08BDBBBB555515
:10544000280000207AF0070808B54FF0AA30194963
:1054500008600846008880B2ADF800000846008861
:1054600080B2ADF80200084600680090042212499C
:105470006846FBF747FC00BF00BF00BF00BF00BF8E
:10548000BFF34F8F00BF00BF00BF0C48006800F49F
:10549000E0600B490843001D0849086000BF00BFD9
:1054A00000BFBFF34F8F00BF00BF00BF00BF00BFF2
:1054B000FDE70000280000207AF007080CED00E06E
:1054C0000000FA0500BF012001F0FEFA012211469A
:1054D0000B48FCF7D3FE0120FCF738FC0022012129
:1054E0000748FCF7CBFEFBF7EFFC06490870FBF71B
:1054F00017FD054908700548FBF748FCE3E7000085
:10550000000C01406000002061000020540F0020CA
:1055100000BF012001F0D8FAFBE700BF012001F035
:10552000D3FAFBE738B502224C496846FBF7D4FBB7
:10553000BDF80200BDF8001040EA0140484908608B
:1055400048480068484908604FF480614748FAF7C6
:1055500082FE474802F04AF841480068B0F1AA3F8D
:1055600008D0B0F1BB3F04D042490844002870D1B4
:105570005BE06FE03B4800683B4908600846016813
:105580003D48FBF7E5F90546E5B137483A49026879
:105590003A4801F069F95020FCF7D8FB38A13348AC
:1055A00000F07CFD0446A2B230493848FEF738FAD4
:1055B00002E00120FCF7CAFB344890F841002128A2
:1055C000F7D016E032A1294800F068FD04465020CB
:1055D00000F0DBFFA2B225492C48FEF721FA02E0D9
:1055E0000120FCF7B3FB294890F841002128F7D0AF
:1055F00038BD1D4801682148FBF7AAF9A0B127A1D1
:105600001A4800F04BFD0446A2B218491F48FEF7A5
:1056100007FA02E00120FCF799FB1C4890F84100D2
:105620002128F7D0FFF7F6FE00BF0F480068B0F55D
:10563000003F0CD20C4801681048FBF789F930B1E3
:10564000002080F3138800BF0C4801F091F901E0BD
:10565000FFE7CDE700BF00BFCAE700007AF0070808
:105660003C0000202400002034000020CC32002028
:10567000004807084544AAAA0000040800000208E0
:105680007570646174696E670000000078470020DF
:10569000636865636B6661696C00000063686563DD
:1056A0006B6F6B0000BF012001F00EFA124800780A
:1056B00001281ED1114800888E281AD11048007880
:1056C00010490978884214D10D484078102810D12B
:1056D0008C210D4800F0C8FE094991F88C10084A49
:1056E00092F88D2041EA0221884202D1FFF7D0FBD7
:1056F000D9E7FEF7E7FFD6E72405002026050020BE
:10570000CC3A002052000020CC32002010B500BF5F
:10571000502080F31188BFF34F8FBFF36F8F00BF0E
:1057200002F0C2FA18B14FF080500449086000BF7F
:10573000002080F3118800BF10BD000004ED00E0E0
:1057400000B595B028210BA8FAF785FD142106A80D
:10575000FAF781FD18216846FAF77DFD01200B90CC
:1057600000040C9000200D9001200F900220129058
:10577000C1031391002114910BA8FDF723F908B17F
:10578000FBF7F5F90F200690022007908020089083
:10579000C000099000200A90002106A8FCF7CCFF69
:1057A00008B1FBF7E4F9022000904003029068463C
:1057B000FCF72AFF08B1FBF7DAF915B000BD704716
:1057C00010B54FF480510348FCF74EFD0248FDF739
:1057D0009EFC10BD000C01408432002010B5024830
:1057E000FDF795FC10BD0000D448002010B50268FC
:1057F000204B98420ED0204B98420BD0B0F1804FF6
:1058000008D01E4B984205D01D4B984202D01D4B2C
:10581000984203D122F070024B681A43154B98420C
:105820000ED0154B98420BD0B0F1804F08D0134BDF
:10583000984205D0124B984202D0124B984203D1A5
:1058400022F44072CB681A4322F080034C6943EA89
:10585000040202608B68C3620B688362054B984246
:1058600002D0054B984201D10B69036301234361C8
:1058700010BD0000002C0140003401400004004035
:1058800000080040000C004030B50C46816821F44F
:105890007F4142EA032525432943816030BD0A4602
:1058A000816821F0700142F007031943816070475D
:1058B00030B50B461446026A056A25F001050562FB
:1058C000816921F0F00141EA041122F00A021A4331
:1058D0008161026230BD30B50B461446026A056A2A
:1058E00025F010050562816921F4704141EA043117
:1058F00022F0A00242EA03128161026230BD70B55B
:1059000005466C6A0020E085E0842046FDF780FDB6
:1059100070BD70B506460025746A20684069C0F302
:10592000C01594F84100212805D125B10020E0845C
:10593000204600F0C8F820684069C0F3801594F84C
:105940004200222805D125B10020E085204600F044
:1059500074F8606C40F0100060642046FDF758FD5C
:1059600070BD70B505466C6A2868006800F02000BC
:10597000002842D1E08500BF00BF21680C3151E80A
:10598000001F21F4807021680C3141E80002002AD8
:10599000F3D100BF00BF00BF2168143151E8001FE0
:1059A00021F001002168143141E80002002AF3D1FE
:1059B00000BF00BF00BF2168143151E8001F21F073
:1059C00040002168143141E80002002AF3D100BFF1
:1059D000202084F84200206B01280ED100BF00BFB8
:1059E00021680C3151E8001F21F0100021680C31B2
:1059F00041E80002002AF3D100BF00206063206B61
:105A0000012804D1A18D2046FDF75BFC02E0204671
:105A1000FDF7A4FF70BD70B505466C6A0120606398
:105A2000206B012805D1A08D41082046FDF749FCD7
:105A300002E02046FDF79AFF70BD00BF00BF02687C
:105A40000C3252E8002F22F4907102680C3242E8C6
:105A50000013002BF3D100BF00BF00BF0268143257
:105A600052E8002F22F001010268143242E80013CC
:105A7000002BF3D100BF016B01290ED100BF00BF85
:105A800002680C3252E8002F22F0100102680C323A
:105A900042E80013002BF3D100BF202180F8421010
:105AA00000210163704710B504462068C06820F0EB
:105AB00040002168C860202084F841002046FDF79E
:105AC000CBFF002010BD00BF00BF02680C3252E8BF
:105AD000002F22F0C00102680C3242E80013002BB4
:105AE000F3D100BF202180F841107047F8B504467B
:105AF00094F84200222875D1A068B0F5805F0CD1DF
:105B0000206950B90025A66A20684068C0F30800E3
:105B10003080A06A801CA06215E0A56A0026A068FB
:105B2000B0F5805F03D0A06828B9206918B9206853
:105B30004068287004E02068406800F07F0028700A
:105B4000A06A401CA062E08D401E80B2E085002863
:105B500046D12068C06820F020002168C860206815
:105B6000C06820F480702168C8602068406920F017
:105B7000010021684861202084F842000020606311
:105B8000206B012826D10020206300BF00BF2168C0
:105B90000C3151E8001F21F0100021680C3141E860
:105BA0000002002AF3D100BF2068006800F0100056
:105BB00010280AD100BF00200090206800680090E3
:105BC00020684068009000BF00BFA18D2046FDF70F
:105BD00078FB02E02046FDF7C1FE0020F8BD01E0A1
:105BE0000020FBE70220F9E770B504462168096947
:105BF00021F44051E2681143226811612269A168D1
:105C00001143626941EA02052168C96841F20C62E8
:105C1000914329432268D1602168496921F4407188
:105C2000A2691143226851612D4A2168914202D133
:105C3000FCF780FE01E0FCF76DFE00EBC00101EB1C
:105C4000001162689200B1FBF2F100EBC00202EBBE
:105C5000001263689B00B2FBF3F26423B2FBF3F221
:105C600002EBC20303EB0212A1EB8201322202EB30
:105C700001116422B1FBF2F101F0F00100EBC0026E
:105C800002EB001263689B00B2FBF3F26423B2FBE9
:105C9000F3F201EB021200EBC00101EB00116368AB
:105CA0009B00B1FBF3F100EBC00303EB001366684C
:105CB000B600B3FBF6F36426B3FBF6F303EBC306BF
:105CC00006EB0313A1EB8301322303EB01116423E1
:105CD000B1FBF3F101F00F0111442268916070BD36
:105CE0000038014077B581B0044615460298A0629D
:105CF000A58500206064222084F842002848E16BDA
:105D000088622848E16BC8622748E16B086300207D
:105D1000E16B486302AE32682368191D2B46E06BC5
:105D2000FBF7C6FF00BF00200090206800680090CD
:105D300020684068009000BF00BF206970B100BFBC
:105D400000BF21680C3151E8001F41F480702168C8
:105D50000C3141E80002002AF3D100BF00BF00BFB0
:105D60002168143151E8001F41F00100216814310D
:105D700041E80002002AF3D100BF00BF00BF216844
:105D8000143151E8001F41F040002168143141E80E
:105D90000002002AF3D100BF002004B070BD000053
:105DA00063590008175A000813590008014691F872
:105DB0004100212828D18868B0F5805F0BD108699F
:105DC00048B90A6A1088C0F308000B685860086A6E
:105DD000801C086205E00B6A581C086218780B6882
:105DE0005860C88C401E80B2C88458B90868C06822
:105DF00020F080000B68D8600868C06840F0400060
:105E00000B68D860002070470220FCE72DE9F041C4
:105E100004460D4617469846069E34E0701C88B32B
:105E20002EB1FCF731FAA0EB0800B0422BD900BF2D
:105E300000BF21680C3151E8001F21F4D0702168A7
:105E40000C3141E80002002AF3D100BF00BF00BFBF
:105E50002168143151E8001F21F00100216814313C
:105E600041E80002002AF3D100BF202084F841005D
:105E700084F8420000BF002084F8400000BF0320E7
:105E8000BDE8F081FFE7206800682840A84201D102
:105E9000012000E00020B842C0D00020F0E7000060
:105EA00008B51C4800680068C0F3001068B300BF64
:105EB00000200090174800680068009015480068AE
:105EC0004068009000BF00BF1248FDF75CFA12481E
:105ED00000684068C0F58060104908800846028864
:105EE0000F491048FAF79EF90C4802880C490E48F1
:105EF000FAF798F94FF4806209490648FDF718FD52
:105F000001200A4908700A4908700248FDF782FA20
:105F100008BD000078470020084800202605002022
:105F2000CC360020CC320020CC3A002024050020C2
:105F30002505002010B50248FDF76CFA10BD0000E1
:105F4000C047002000BFFEE72DE9F04705460F4699
:105F500090460024284600F021FBFBF7C5FF41488E
:105F600085420CD117F80840224600230146012043
:105F7000FBF762FF06460EB93B4804806EE03B48E3
:105F800085420CD117F80840224600230146012023
:105F9000FBF752FF06460EB935490C705EE03548F6
:105FA00085420CD117F80840224600230146012003
:105FB000FBF742FF06460EB92F4804804EE02F48FB
:105FC000854202D02E48854248D14FF43A762B487C
:105FD00085421FD12B480088B04204DB2948008845
:105FE000801B84B205E027480088301A84B244F44C
:105FF00000442246002321490120FBF71DFF814672
:10600000B9F1000F05D1C4F30E001F4908801F48E5
:10601000048022E01A4885421FD11D480088B04202
:1060200004DB1B480088801B84B205E01848008808
:10603000301A84B244F4004422460023104901205F
:10604000FBF7FAFE8146B9F1000F05D1C4F30E004B
:10605000104908801048048000BF00BFFBF7E2FE33
:10606000BDE8F0870000070852000020000807087C
:1060700061000020001007085400002000180708E5
:106080000020070882000020860000207400002005
:106090008400002088000020760000200FB4084B08
:1060A00010B504A902AA039800F038F8044602A922
:1060B000002000F0D4F9204610BC5DF814FB00006D
:1060C0005F64000802480068C0F3022070470000C7
:1060D0000CED00E010B5002804DB0A07130E054A9A
:1060E000135406E00A07140E034A00F00F031B1FA7
:1060F000D45410BD00E400E018ED00E002E008C850
:10610000121F08C1002AFAD170477047002001E031
:1061100001C1121F002AFBD1704700002DE9FF4F7B
:106120008BB088460546002606E025280BD0DDE921
:106130000D1290476D1C761C28780028F5D10FB001
:106140003046BDE8F08F0024A146A2460122AE49A8
:1061500000E0044315F8013F203B02FA03F0084237
:10616000F7D128782A2810D06FF02F022878A0F1D4
:106170003001092915D809EB890102EB410144F0EE
:10618000020400EB01096D1CF0E758F8041B5FEAFC
:10619000010903D544F40054C9F1000944F0020494
:1061A0006D1C28782E2817D115F8010F44F004042F
:1061B0002A280ED06FF02F022878A0F1300109298B
:1061C0000AD80AEB8A0102EB410100EB010A6D1CBF
:1061D000F2E758F804AB6D1C28786C280FD006DC69
:1061E0004C2817D068280DD06A2814D104E07428F0
:1061F00010D07A280FD10DE044F400140AE044F4E2
:10620000801401E044F440146978814202D104F51D
:1062100080146D1C6D1C2878692865D006DC002868
:106220008DD0632827D0642806D15DE06E2808D081
:1062300073282AD0752877D0DDE90D129047761C97
:10624000E0E0C4F30250022809D003280DD0D8F8AA
:10625000001004280DD00E6008F10408D2E0D8F830
:106260000010F217C1E90062F6E7D8F800100E80BE
:10627000F2E70E70F0E718F8041B8DF8001000200C
:106280008DF80100EB46012003E058F804BB4FF005
:10629000FF3061074FF0000701D40AE07F1C57452B
:1062A0000DDA8742FADB1BF807100029F6D106E069
:1062B0007F1C8742FCDB1BF807100029F8D1DDE9C1
:1062C0000D23A9EB07008146214600F0B1F83044C8
:1062D000C61904E0DDE90D121BF8010B90477F1E83
:1062E000F8D22146484688E058F8040BC4F302511E
:1062F0004FF00A0B032900D100B2042900D140B2AB
:10630000002802DA40422D2102E0210505D52B218B
:106310008DF82410012104E006E0E10710D02021CF
:10632000F6E708AF089113E058F8040BC4F30251E4
:106330004FF00A0B032900D180B2042900D1C0B26A
:106340000021EEE75946FAF751F9303107F8011DFF
:106350000028F7D1ADEB070000F1200B600702D554
:1063600024F4803401E04FF0010ADA4502DDAAEBA3
:106370000B0000E00020824600EB0B01089801446E
:10638000A9EB01000A90E00306D4DDE90D232146C4
:106390000A9800F04DF806444FF0000908E009A9FA
:1063A00011F80900DDE90D12904709F10109761C89
:1063B00008998945F3DBE0030CD5DDE90D2321467F
:1063C0000A9800F035F8064404E0DDE90D123020AB
:1063D0009047761CBAF10001AAF1010AF5DC05E04C
:1063E000DDE90D1217F8010B9047761CBBF1000197
:1063F000ABF1010BF4DC0A982146DDE90D2300F036
:1064000005F806446D1C97E6092801002DE9F041C6
:10641000044600251E461746880404D405E0394684
:106420002020B0476D1C641EF9D52846BDE8F081D8
:106430002DE9F041044600251E469046C80301D5CB
:10644000302700E02027880404D505E0414638467F
:10645000B0476D1C641EF9D52846BDE8F0810A6876
:10646000531C0B601070704730B502460B464FF658
:10647000FF70002110E0545C6040002409E000F04F
:10648000010525B14AF2010585EA600000E04010EF
:10649000641C082CF3DB491C9942ECDB30BD000086
:1064A00010B504460B480068C06820F40050094944
:1064B0000968C86007484460FDF71EF908B1FAF79B
:1064C00056FB04480068C06840F400500149096860
:1064D000C86010BD7847002010B54FF480610748B0
:1064E000F9F7B9FE4FF480610548F9F7B4FE0020D2
:1064F000044908700449087010BD0000CC3A00201F
:10650000CC360020250500202405002010B5028887
:10651000C2F30323027863F31F1213064288C2F307
:10652000032464F31F1243EA02438288C2F3032464
:1065300064F31F1243EA0223C288C2F3032464F304
:106540001F1213430B6010BD30B502460B460020EE
:10655000002117E0545C80EA042000240EE000F4DF
:1065600000452DB141F2210585EA4005A8B203E0BE
:106570004FF6FF7505EA4000651CECB2082CEEDB17
:106580004C1CA1B29942E5DB30BDC200002100BF26
:1065900001E000BF491C9142FBD3704730B585B084
:1065A00004460020019003940120049000200090F4
:1065B000FBF79AFC694601A8FBF7DCFB0546FBF7F5
:1065C00031FC15BB1248844203D1002011490880D8
:1065D0001BE01148844203D100201049087014E0E8
:1065E0000F48844204D14FF6FF700E4908800CE03A
:1065F0000D48844203D100200C49088005E00C4876
:10660000844202D100200B49088005B030BD000053
:106610000000070852000020000807086100002061
:10662000001007085400002000180708860000200A
:1066300000200708880000202DE9FF4F8BB08B4613
:1066400090469946199E0020089009F1010258F8D9
:10665000221058F82900F9F762FE82466649F9F7D8
:1066600096FE07900A960A9EB00000F0F7F90446DD
:106670004FF0000A12E05046F9F739FF03900799EE
:10668000F9F753FE049009F1010058F8201004981E
:10669000F9F7F3FD44F82A000AF1010AB245EADBF2
:1066A0004FF0FF35554806904FF0000A22E054F8AD
:1066B0002A100B98F9F733FE0190F9F753FF21F0F8
:1066C0000041CDE90201F9F760FF049006990498B2
:1066D000F9F778FF01D2504600E0284605460699B2
:1066E0000498F9F76FFF01D2049800E0069806902D
:1066F0000AF1010AB245DADB414805900996099E84
:10670000B00000F0ABF907464FF0000A11E0504628
:10671000F9F7EDFE3A490390F9F707FE049018984F
:106720005BF820100498F9F7A8FD47F82A000AF151
:10673000010AB245EBDB54F825003249F9F74CFF6A
:1067400004D248F29010304908804AE054F82500FD
:106750002E49F9F741FF1FD254F825002949F9F7CE
:1067600031FF19D857F82500F9F7FCFE21F0004158
:106770000022274BCDE90001F9F747FECDE90201E0
:10678000F9F7D7FE80B20890089840F400400890CE
:106790001D490898088024E054F825001D49F9F7A0
:1067A0001BFF10D854F825001849F9F70BFF0AD839
:1067B00057F825001049F9F7B8FD8246F9F7A5FE0C
:1067C000114908800DE054F825001249F9F7FAFE46
:1067D00004D240F21A400C49088002E000200A4925
:1067E000088000200890384600F016F8204600F097
:1067F00013F80FB0BDE8F08F0000204100007A448C
:10680000CDCCCC3DB57DAA4320050020E9F702425E
:10681000000024408104153F10B5002821D0114B01
:106820000022001F196803E0814203D80A46496824
:106830000029F9D152B11368841A9C4204D100682E
:1068400018441060104602E0506000E0186039B152
:1068500002680B1A934203D10B681A44026049681C
:10686000416010BD100600202DE9FC4781460C4612
:106870001546AFB2264632483249086007F5006037
:10688000C11700EB5151C9122F4A11804FF400611A
:106890002E48F9F7E0FC2EA103C9CDE90001012043
:1068A0002D49086044E0012211462C48FBF7E6FC24
:1068B0000520FBF74BFA002201212848FBF7DEFCFC
:1068C0004FF4006231462148FAF706FA4FF480622D
:1068D0001C4801681D48FAF715FA5020FFF755FECD
:1068E0001D486A461EA103681F48FFF7D7FB804674
:1068F0001FFA88F21C491D48FDF792F806F500665C
:106900001048006800F500600E4908600122114639
:106910001248FBF7B3FC0520FBF718FA002201210F
:106920000E48FBF7ABFC0C480068401C0A490860A5
:1069300009480068044909888842B4DDBDE8FC873D
:106940000000020844000020400000200020002039
:1069500061636B3D0000000048000020000C014016
:10696000257325640D0A0000CC32002078470020F2
:1069700070B5044672B6206880F3088800BF656869
:10698000A84770BDFBF792FCFEF7DAFEFDF7A0FD0D
:10699000FDF736FDFDF75CFEFDF7ECFCFDF720FE94
:1069A000FDF772FE1E48FCF7E3FA1E4800F01EFEDB
:1069B000FEF7B8FDF9F78EFF1B4800F07BFE1A4882
:1069C0000E3000F049FE194800F0D4FB184800F0E2
:1069D000CDFB054600F0BEFD164800F0C7FB05469E
:1069E00000F0EEFD14A11648FFF758FB0446A2B2D2
:1069F00013491448FDF714F84FF480621249114806
:106A0000FCF796FF0F480068C06840F010000D4981
:106A10000968C860FDF71EFD00F062F800BFFEE7E0
:106A200084320020004807087AF0070800000708B1
:106A300000080708001007086170703100000000AE
:106A4000CC32002078470020CC36002001460020C0
:106A5000842901D0CA1C104470470000F0B50B30E7
:106A6000154D20F007010024144A0FE003688B4203
:106A70000BD38B4205D95E1A43184768C3E90067F8
:106A800000E04368136002C004E0021D10680028A3
:106A9000ECD12046002802D1286808B10020F0BDC2
:106AA000064A07481060074A121A22F00702C0E996
:106AB000002401202860D7E71406002010060020DB
:106AC000145600201058002070B5044625460DB11C
:106AD000294600E00121084600F008FF002070BDB3
:106AE00010B500F031FF002010BD7FB504460D4603
:106AF000606998B1A06988B1B4F90800FFF7A6FFF2
:106B00000646D4E90510CDE9006102902B462269C2
:106B1000D4E9001001F06CF8039013E0B4F9080018
:106B2000FFF794FF064603A8CDE90060238A9AB2D6
:106B30002B46D4E9001001F029F8012802D00020EA
:106B400004B070BD0398FBE72DE9F04105460E4601
:106B50001C4807681C480068001D00F0CBFD50B9B8
:106B60001948006890F82C100120884017490968DE
:106B7000814316480160681C38B936B11248016873
:106B8000091D134800F000FE1AE07C190E48006849
:106B90004460BC4207D20C480168091D0D480068DA
:106BA00000F0D8FD0CE008480168091D0A4800689B
:106BB00000F0D0FD09480068844201D20748046013
:106BC000BDE8F081C4050020B0050020C805002004
:106BD000F8490020B8050020B4050020E005002099
:106BE00010B5044600F0DCFD23480068401C224933
:106BF00008602248006840B92048046008460068E0
:106C000001280DD100F03AF90AE01D48006838B9B2
:106C10001A480068C06AE16A884201D817480460CF
:106C200018480068401C1749086094F82C1001208F
:106C3000884015490968084313490860E16A01EB77
:106C40008101124A02EB8100211D00F09DFD00F040
:106C5000D1FD0B48006868B108480068C06AE16A65
:106C6000884207D24FF0805009490860BFF34F8F28
:106C7000BFF36F8F10BD0000C0050020B0050020DD
:106C8000CC050020DC050020C80500201C490020A0
:106C900004ED00E010B516E000F082FD0C48C0687D
:106CA000C468201D00F026FD0A480068401E0949FE
:106CB000086009480068401E0749086000F09AFD16
:106CC000204600F00BF8044800680028E4D110BD0D
:106CD000E4490020C0050020BC05002010B5044692
:106CE00094F8510030B9206B00F0A2FD204600F06E
:106CF0009FFD1AE094F85100012803D1204600F0CE
:106D000097FD12E094F85100022801D1012000E023
:106D1000002050B900BF502080F31188BFF34F8F7F
:106D2000BFF36F8F00BF00BFFEE710BD30B54FF45B
:106D30004063174800F007042CB1C01D20F0070085
:106D4000134C041B1B1B0246124C22600024114DE5
:106D50006C60D018083820F007000F4C2060002429
:106D60000D4D2D686C600C4D2D682C601146441A39
:106D70004C60094C24680C60084D4C682C60084D30
:106D80004C682C604FF00044064D2C6030BD000074
:106D90000C4A0020EC050020F4050020FC05002032
:106DA000F80500200006002000BFFFF773FF06482B
:106DB00000680128F9D94FF0805004490860BFF3FA
:106DC0004F8FBFF36F8FF0E71C49002004ED00E008
:106DD0002DE9FF5F81460F469246DDE90E6B109C60
:106DE000AAF10100216B01EB800828F0070808F0E8
:106DF000070008B9012000E0002050B900BF502072
:106E000080F31188BFF34F8FBFF36F8F00BF00BFB8
:106E1000FEE7002507E0795D04F134004155785D17
:106E200000B902E06D1C102DF5D300BF00214320F6
:106E30000155072E00D30626E66266640020A06492
:106E4000201D00F084FC04F1180000F080FC246197
:106E5000C6F10700A06164620020E06484F850007D
:106E600049464046039A00F049F92060BBF1000F03
:106E700001D0CBF80040BDE8FF9F000010B5002412
:106E800007E004EB84010F4A02EB810000F052FCA2
:106E9000641C072CF5D30C4800F04CFC0B4800F0A8
:106EA00049FC0B4800F046FC0A4800F043FC0A4845
:106EB00000F040FC0448094908600448084908609B
:106EC00010BD00001C490020A8490020BC4900203A
:106ED000D0490020E4490020F8490020B4050020F2
:106EE000B805002010B50146164800E000680368A8
:106EF0008B42FBD30246436813448B4204D1436860
:106F00004C682344436001460A464B6813440468B6
:106F1000A34211D10C4C03682468A34208D04B68EB
:106F20000468646823444B6003681B680B6005E0D9
:106F3000054B1B680B6001E003680B60884200D0C2
:106F4000016010BDEC050020F40500200A49096825
:106F5000096809B9012100E0002121B14FF0FF319A
:106F6000064A116006E004490968C968C868034A0E
:106F70004168116070470000B4050020E005002062
:106F80000E480068401C08B9012000E0002050B9FC
:106F900000BF502080F31188BFF34F8FBFF36F8F76
:106FA00000BF00BFFEE700BF502080F31188BFF391
:106FB0004F8FBFF36F8F00BF00BFFEE704060020B6
:106FC0002DE9F04104464FF0000800F015FD464859
:106FD000006808B9FFF7AAFE44480068204000286E
:106FE0006BD1D4B1083404F00700B0B104F007004D
:106FF000C0F10800044404F0070008B9012000E0D3
:10700000002050B900BF502080F31188BFF34F8F8C
:10701000BFF36F8F00BF00BFFEE7002C4DD0344898
:107020000068844249D8334E3046056801E02E4658
:107030002D686868A04202D228680028F7D12A4843
:107040000068854239D0306800F10808286830604F
:107050006868001B102819D92F1907F0070008B914
:10706000012000E0002050B900BF502080F31188BB
:10707000BFF34F8FBFF36F8F00BF00BFFEE768689D
:10708000001B78606C603846FFF72CFF1849686871
:107090000968081A16490860084600681649096810
:1070A000884203D212480068134908600F49686893
:1070B0000968084368600020286000F099FE08F025
:1070C000070008B9012000E0002050B900BF50209F
:1070D00080F31188BFF34F8FBFF36F8F00BF00BFE6
:1070E000FEE74046BDE8F081F405002000060020E0
:1070F000F8050020EC050020FC050020001F4FF0E3
:1071000080730360001F21F001030360001F034B25
:10711000036014380260203870470000816F000857
:1071200010B50548FCF7CEF84FF4806203490248D9
:10713000FCF7FEFB10BD000078470020CC36002095
:1071400002460948006838B1002002E00B5C135485
:10715000401C0528FADB06E0002002E00B5C13541B
:10716000401C0428FADB70473000002001460888E4
:107170007047000010B504462046FFF7F7FF0346AE
:107180004FF6FF70834204D103480088024908800B
:1071900001E00148038010BD520000202DE9FE4FA0
:1071A00006460F4690461D46DDE90C9A0E9C0020CF
:1071B000009001900290F0B28DF800008DF80170FF
:1071C0008DF8028028128DF80300E8B28DF80400D3
:1071D0004FEA29208DF8050009F0FF008DF8060020
:1071E0004FEA2A208DF807000AF0FF008DF808000A
:1071F000A01EC1B26846FFF737F983460BF0FF01C6
:10720000A01E0DF800104FEA2B21601E0DF8001093
:10721000631EA2B269460448FCF7A9FBFFF75CF9BC
:10722000FFF77EFFBDE8FE8F784700202DE9F04F85
:1072300085B006460F4690461D46DDE90FABDDF8EA
:107240003890119C00200190029003900490F0B2BD
:107250008DF804008DF805708DF8068028128DF8E1
:107260000700E8B28DF808004FEA29208DF80900E0
:1072700009F0FF008DF80A004FEA2A208DF80B0074
:107280000AF0FF008DF80C004FEA2B208DF80D005E
:107290000BF0FF008DF80E00A01EC1B201A8FFF791
:1072A000E3F800900098C1B2A01E01AA1154009802
:1072B0000112601E1154631EA2B201A90448FCF71A
:1072C00056FBFFF709F9FFF72BFF05B0BDE8F08F7C
:1072D000784700202DE9F04F85B006460F469046CE
:1072E0001D46DDE911B4DDE90E9A002001900290FF
:1072F00003900490F0B28DF804008DF805708DF8BD
:10730000068028128DF80700E8B28DF808004FEAD1
:1073100029208DF8090009F0FF008DF80A004FEAD6
:107320002A208DF80B000AF0FF008DF80C00109851
:1073300000128DF80D001098C0B28DF80E004FEAC3
:107340002B208DF80F000BF0FF008DF81000A01E11
:10735000C1B201A8FFF788F800900098C1B2A01E42
:1073600001AA115400980112601E1154631EA2B2AA
:1073700001A90548FCF7FBFAFFF7AEF8FFF7D0FECE
:1073800005B0BDE8F08F0000784700202DE9FC47EC
:1073900006460F4690461D460A9C0020009001902C
:1073A000F0B28DF800008DF801708DF8028028127F
:1073B0008DF80300E8B28DF80400A01EC1B2684643
:1073C000FFF752F8814609F0FF01A01E0DF80010EA
:1073D0004FEA2921601E0DF80010A2B2234669462B
:1073E0000448FCF7C4FAFFF777F8FFF799FEBDE809
:1073F000FC870000784700202DE9FC4107468846BD
:1074000014461D46002000900190F8B28DF800004F
:107410008DF8018020128DF80200E0B28DF8030093
:1074200028128DF80400E8B28DF8050006216846A0
:10743000FFF71AF80646F0B28DF8060030128DF804
:1074400007000723082269460448FCF790FAFFF773
:1074500043F8FFF765FEBDE8FC8100007847002097
:107460002DE9FE4F06460F4690461D46DDE90C9479
:107470000020009001900290F0B28DF800008DF88D
:1074800001708DF8028028128DF80300E8B28DF8A3
:1074900004004FEA29208DF8050009F0FF008DF85F
:1074A0000600A01EC1B26846FEF7DEFF82460AF063
:1074B000FF01A01E0DF800104FEA2A21601E0DF8F2
:1074C0000010631EA2B269460448FCF750FAFFF7A9
:1074D00003F8FFF725FEBDE8FE8F00007847002087
:1074E0002DE9FE4306460F4614461D46DDF828905A
:1074F0000020009001900290F0B28DF800008DF80D
:10750000017020128DF80200E0B28DF803002812FD
:107510008DF80400E8B28DF805008DF8069007217B
:107520006846FEF7A1FF804608F0FF008DF80700CF
:107530004FEA28208DF8080009231A4669460448B6
:10754000FCF715FAFEF7C8FFFFF7EAFDBDE8FE837A
:107550007847002010B504464FF6FF70844214D1DE
:10756000002208211548FAF789FE0022102113484D
:10757000FAF784FE002220211048FAF77FFE00224D
:1075800040210E48FAF77AFE17E004F001020821C4
:107590000A48FAF773FEC4F3400210210748FAF7CD
:1075A0006DFEC4F3800220210448FAF767FEC4F39D
:1075B000C00240210148FAF761FE10BD000C0140F5
:1075C00010B50446072C04DC074951F82400FEF7E7
:1075D00067FF4FF6FF70844201D0032C03D14FF4B4
:1075E0001650FEF75DFF10BD4005002010B50446A3
:1075F000022221461648F9F76FFB00200FE01449DC
:1076000031F810104FF47F4202EA0121104A32F89B
:10761000102041EA12210E4A22F81010401C0128C5
:10762000EDDB0B4800884FF6FF71884203D1002044
:10763000084908600BE0064800884FF47F4101EAE2
:1076400000200349098840EA11200249086010BD62
:10765000380500202400002038B5044608221249CD
:107660001248F9F739FB00200FE0104931F81010EB
:107670004FF47F4202EA01210C4A32F8102041EA1D
:1076800012210A4A22F81010401C0428EDDB69463A
:107690000648FEF73BFF0098401C00B938BD04497E
:1076A0000098086000BFF9E788F00708060000208E
:1076B0005800002010B5044610220C490C48F9F778
:1076C0000BFB00200FE00A4931F810104FF47F4205
:1076D00002EA0121064A32F8102041EA1221044A46
:1076E00022F81010401C0828EDDB10BD00500708E0
:1076F0007A06002001460A69D1E901309860D1E993
:10770000010358605068884201D1886850600020A9
:1077100008611068401E106010687047034B0360DA
:10772000034B0B6080231360704700003030002053
:107730008430002000F1080141604FF0FF3181608A
:1077400000F10801C1600161002101607047002162
:107750000161704710B502460B685C1C0CB91069DA
:1077600007E002F1080000E04068446824689C4299
:10777000FAD944684C604C68A160886041600A6135
:107780001468641C146010BD42684A6093688B6082
:10779000936859609160086103685B1C03607047DF
:1077A00000BF502080F31188BFF34F8FBFF36F8F5E
:1077B00000BF0E480068401C0C490860084600687D
:1077C000012812D10A480068C0B208B9012000E0BF
:1077D000002050B900BF502080F31188BFF34F8FB5
:1077E000BFF36F8F00BF00BFFEE7704704060020A5
:1077F00004ED00E00D48006850B900BF502080F350
:107800001188BFF34F8FBFF36F8F00BF00BFFEE73C
:1078100006480068401E054908600846006820B90F
:10782000002080F3118800BF00BF704704060020CD
:1078300070B506463546002E3FD0083D2C461F4900
:1078400060680968084008B1012000E0002050B9D4
:1078500000BF502080F31188BFF34F8FBFF36F8FAD
:1078600000BF00BFFEE7206808B9012000E000204B
:1078700050B900BF502080F31188BFF34F8FBFF382
:107880006F8F00BF00BFFEE70C49606809680840C1
:1078900098B1206888B909496068096888436060C0
:1078A00000F0AAF8064960680968084404490860BD
:1078B0002046FFF717FB00F09BFA70BD0006002082
:1078C000F805002000204FF0E0210861886106489B
:1078D00000684FF47A71B0FBF1F0401E4FF0E021E8
:1078E0004861072008617047AC05002070B5044668
:1078F0000025D4B11248006808B9012000E000203A
:1079000050B900BF502080F31188BFF34F8FBFF3F1
:107910006F8F00BF00BFFEE700F06EF80021204629
:10792000FFF712F900F064FA05463DB94FF08050B8
:1079300004490860BFF34F8FBFF36F8F70BD000025
:10794000E805002004ED00E010B586B000200590A9
:10795000049003AA04A905A8FFF7E0FE0022DDE9D0
:1079600004101346CDE9002102901CA11D48039A82
:1079700000F03EF91C4908600846006808B101247F
:1079800000E00024012C15D100BF502080F31188A5
:10799000BFF34F8FBFF36F8F00BF4FF0FF3013491E
:1079A000086001201249086000201249086000F0B8
:1079B00071F810E0601C08B1012000E0002050B90F
:1079C00000BF502080F31188BFF34F8FBFF36F8F3C
:1079D00000BF00BFFEE706B010BD000049444C45A3
:1079E00000000000A96D0008E4050020E00500206B
:1079F000CC050020C405002002480068401C014955
:107A000008607047E80500201D48006818B1012093
:107A10001C49086032E000201A4908601A480068D2
:107A2000B0FA80F0C0F11F0101EB8100174A52F853
:107A3000200008B1012000E0002050B900BF502014
:107A400080F31188BFF34F8FBFF36F8F00BF00BF6C
:107A5000FEE701EB81020D4B03EB820042685268A6
:107A6000426000F108024368934202D142685268C2
:107A700042604268D268064B1A6000BF704700003F
:107A8000E8050020D4050020C80500201C4900207E
:107A9000B00500201CB53849084600780190FF2049
:107AA0000A4610700846007800909DF8000000F02B
:107AB000F0009DF80020904201D1012000E000205C
:107AC00050B900BF502080F31188BFF34F8FBFF330
:107AD0006F8F00BF00BFFEE79DF8000000F0500070
:107AE000264A10700720264A106009E024480068E2
:107AF000401E234A10609DF800004006000E0090D2
:107B00009DF8000000F080008028EFD01C4800683D
:107B1000C0F10700042801D1012000E0002050B985
:107B200000BF502080F31188BFF34F8FBFF36F8FDA
:107B300000BF00BFFEE7124800680002104A106054
:107B40001046008800F4E06010600B4A0198107045
:107B50000C48006840F470000A4908600846006854
:107B600040F070400860FFF7ADFE00200649086055
:107B7000F8F7FCFA00201CBD00E400E00806002035
:107B80000C06002020ED00E0040600202DE9FF4F48
:107B900085B0804689461746DDE912ABB800FFF78D
:107BA0000FFA064656B15420FFF70AFA04460CB104
:107BB000266304E03046FFF73BFE00E000248CB172
:107BC000002084F85100CDE900ABCDE902403A46EF
:107BD00049464046089BFFF7FBF82046FFF700F8B0
:107BE000012501E04FF0FF35284609B0BDE8F08FD0
:107BF0002DE9F04F85B00746884691469A46DDE963
:107C00000EB6109C0EB1012000E0002050B900BF5C
:107C1000502080F31188BFF34F8FBFF36F8F00BFE9
:107C200000BFFEE70CB1012000E0002050B900BF0A
:107C3000502080F31188BFF34F8FBFF36F8F00BFC9
:107C400000BFFEE7542003900398542801D101207F
:107C500000E0002050B900BF502080F31188BFF32E
:107C60004F8FBFF36F8F00BF00BFFEE7B4B1AEB15F
:107C700025462C462E63022085F85100002004A9D9
:107C800053464A46CDE900B1CDE902504146384657
:107C9000FFF79EF82846FEF7A3FF01E000200490BE
:107CA000049805B0BDE8F08F2DE9F0414FF00008D1
:107CB00044480068002877D143480068451C424882
:107CC000056015BB41480068006808B9012000E064
:107CD000002050B900BF502080F31188BFF34F8FB0
:107CE000BFF36F8F00BF00BFFEE738480768384812
:107CF0000068364908603648076036480068401C0E
:107D000034490860FFF722F900BF33480068854214
:107D10003CD300BF2D480068006808B9012000E08E
:107D2000002020B14FF0FF302B4908602DE027489C
:107D30000068C068C4686668B54202D2264806601A
:107D400023E0201DFFF7D6FCA06A18B104F118004B
:107D5000FFF7D0FC94F82C10012088401F490968D7
:107D600008431E490860E16A01EB81011C4A02EBED
:107D70008100211DFFF708FD1A49E06A0968C96AF8
:107D80008842C7D34FF00108C4E700BF1548006818
:107D9000C06A00EB8000124951F82000012801D987
:107DA0004FF0010805E0FFE70F480068401C0E494E
:107DB00008600E48006808B14FF001084046BDE871
:107DC000F0810000E8050020C4050020B405002073
:107DD000B8050020D8050020E0050020C8050020D7
:107DE0001C490020B0050020D0050020D40500204B
:107DF00070B5002400263648006850B900BF5020F6
:107E000080F31188BFF34F8FBFF36F8F00BF00BFA8
:107E1000FEE7FFF7C5FC2E480068401E2C490860AD
:107E20000846006800284FD12A48006800284BD037
:107E300024E02948C068C46804F11800FFF75AFC20
:107E4000201DFFF757FC94F82C100120884023498F
:107E50000968084321490860E16A01EB8101204A71
:107E600002EB8100211DFFF78FFC1E49E06A0968C3
:107E7000C96A884202D301201B490860164800687D
:107E800008B9012000E000200028D2D00CB1FFF793
:107E90005DF81648056865B100BFFFF705FF10B132
:107EA0000120114908606D1E002DF6D100200F49F8
:107EB00008600D48006838B1012630070C49086099
:107EC000BFF34F8FBFF36F8FFFF794FC304670BD49
:107ED000E8050020C0050020D0490020C80500208A
:107EE0001C490020B0050020D4050020D00500204A
:107EF00004ED00E00008014001000000000801401E
:107F000002000000000801400400000000080140D9
:107F100008000000000801401000000000080140B7
:107F2000200000000008014040000000000801405F
:107F30008000000004800008A5560008030000002F
:107F400000000000800000000000000000000000B1
:107F5000E07F0008C5540008030000000000000096
:107F6000800000000000000000000000EC7F00081E
:107F70001155000803000000000000008000000010
:107F80000000000000000000F87F00081B550008FA
:107F9000030000000000000080000000000000005E
:107FA0000000000002030405060708090A0B0C0D77
:107FB0000E0F1010010202030405060708090A0B40
:107FC0000C0D0E0F10100102000000000000000058
:107FD000010203040607080900000000010203046F
:107FE0006D795461736B3032000000006D7954611B
:107FF000736B3033000000006D795461736B303463
:10800000000000006961705461736B002C800008EF
:1080100000000020180600008207000860840008A5
:1080200018060020F85500000C6100080122032EFC
:10803000040862C104320708232320C21A1C041A50
:1080400018041A14041A10041A0C041A08041A0446
:10805000041119041AF8611AF0041AE8041AE00469
:108060001AD8041AD0041AC8041AC0041AB8041A78
:10807000B0041AA8041AA0041A98041A90041A88C2
:10808000041A80041A70041A60041A50041A400476
:108090001A30041A20042A10B929541AC0481904A5
:1080A0001AA0041A80041A400411290C62BF3380FC
:1080B0003F1A400319041A80041AA0041AC0041AB3
:1080C000E004111A414819041A20041A30041A4015
:1080D000041A50041A60041A70041A80041A8804DE
:1080E0001A90041A98041AA0041AA8041AB0041AC0
:1080F000B8041AC0041AC8041AD0041AD8041AE022
:10810000041AE8041AF0041AF8041122421A0404AA
:108110001A08041A0C041A10041A14041A18041A5F
:108120001C041A20041A24041A28041A2C041A30D5
:10813000041A34041A38041A3C041A40041A440479
:108140001A48041A4C041A50041A54041A58041AEF
:108150005C041A60041A64041A68041A6C041A7025
:10816000041A74041A78041A7C041A80041A82040B
:108170001A84041A86041A88041A8A041A8C041AA7
:108180008E041A90041A92041A94041A96041A98E7
:10819000041A9A041A9C041A9E041AA0041AA2042F
:1081A0001AA4041AA6041AA8041AAA041AAC041AD7
:1081B000AE041AB0041AB2041AB4041AB6041AB8F7
:1081C000041ABA041ABC041ABE041AC0041AC2045F
:1081D0001AC4041AC6041AC8041ACA041ACC041A07
:1081E000CE041AD00400FF00D242CC76AA434870D5
:1081F0009F43EB32954324AF8B43A5D68243A138EE
:1082000075433EE8654318A65743D95D4A43E0FCF1
:108210003D4313723243A5AD274313A11D43FA3EDC
:1082200014430F7B0B43EF4903434142F742FAEDFE
:10823000E8421F85DB423FF7CE421835C3427D300E
:10824000B8426ADCAD42E72CA442A1169B42428FA1
:108250009242438D8A42A107834271EC774282A207
:108260006A4254235E42B16152424E514742B5E6E2
:108270003C423F17334217D92942EB2221423DECC1
:1082800018420E2D114201DE0942E9F7024210E9BF
:10829000F841719BEC41B3FBE0412EFFD541439C7B
:1082A000CB4186C9C141917EB84133B3AF41D95F5B
:1082B000A741BF7D9F41F00598417CF29041713DFF
:1082C0008A41B1E1834168B37B41F2417041666606
:1082D000654159175B41D34D51410C0248410E2D68
:1082E0003F414BC8364120099FCD2E414C37274195
:1082F0001015204168221941029A12417C610C41FB
:108300008E750641B7D118F9418FE4F6401EA7ECEF
:10831000408FE4E2405396D940AEB6D040143FC8F7
:10832000406B2BC040C976B840A01AB1407B14AA5C
:10833000409E5EA340C3F59C40D0D596407FFB9005
:1083400040B7628B40D50986401CEB80401B0D78FE
:10835000407DAE6E4017B76540A3235D40EEEB5401
:1083600040B30C4D404D8445408C4A3E40705F37D1
:10837000400EBE30407C612A4017482440986E1E53
:10838000405BD318407671134045470E4083510936
:10839000408A8E044072F9FF3F9031F73F27C2EECA
:1083A0003FA9A4E63F5DDCDE3F705FD73FE02DD004
:1083B0003F2041C93F3199C23FCA32BC3FA60AB6ED
:1083C0003F7E1DB03F0A68AA3F4BEAA43FF9A09F39
:1083D0003FCE889A3FCBA1953FA7E8903F1D5A8C8E
:1083E0003F72F9873F1AC0833F9B557F3FA779773C
:1083F0003F57EC6F3F029A683FC58F613F83C05A79
:1084000048003310543F0DE04D3FBEC1473FDCD71D
:10841000413FF6283C3FF0A7363FCA54313F113662
:108420002C3FAB3E273F2575223FF2D21D3F10580F
:10843000193F8104153F5AFF01C123B0042360098D
:1084400023C012338025324B329632E113C201022F
:10845000438032104201035524F41AAA010110008E
:0400000508000131BD
:00000001FF
